:101C3800616D706C2025660020002A2A2000202A69
:101C48002A00202020416464726573733A2020259D
:101C58003034580020205265766973696F6E3A20D7
:101C6800202573004F76657263757272656E7420F5
:101C78003E302E3541206F6E002020202035562022
:101C88006F75747075742021212120202000202078
:101C9800204F76657263757272656E74206F6E2060
:101CA800202000202020323456206F7574707574FF
:101CB8002021212120202000524553455420202056
:101CC80020202020202020202020202000506C656B
:101CD80061736520696E73657274206D6F64756CCD
:101CE800650020202744494E203556272028307883
:101CF8003230292020200020202020696E746F2097
:101D0800706F72742035202020202000457874657B
:101D1800726E616C205472696767657200467265FD
:101D28007175656E63793A2025642000487A202011
:101D380020006B487A202020004D487A202020007F
:101D4800416D706C69747564653A2025626420255C
:101D58002520202000202D20487A202B20202020FC
:101D6800202D20416D70202B004C45442050554CAF
:101D7800534552002449643A207363735F3230300C
:101D8800302E63203238373420323030352D31311F
:101D98002D31352030383A34373A31345A20726987
:101DA800747420240001340000004672657100003C
:101DB800000001003900419000003F800000000051
:101DC8000000000000013400000050576964746886
:101DD800000001003A0141A000003F80000000001F
:101DE8000000000000045D000001416D706C30309F
:101DF800000001003C0042C800003F8000000000D5
:101E08000000000000045D000001416D706C30317D
:101E180000000100400042C800003F8000000000B0
:101E28000000000000045D000001416D706C30325C
:101E380000000100440042C800003F80000000008C
:101E48000000000000045D000001416D706C30333B
:101E580000000100480042C800003F800000000068
:101E68000000000000045D000001416D706C30341A
:101E7800000001004C0042C800003F800000000044
:101E88000000000000045D000001416D706C3035F9
:101E980000000100500042C800003F800000000020
:101EA8000000000000045D000001416D706C3036D8
:101EB80000000100540042C800003F8000000000FC
:101EC8000000000000045D000001416D706C3037B7
:101ED80000000100580042C800003F8000000000D8
:101EE8000000000000045D000001416D706C303896
:101EF800000001005C0042C800003F8000000000B4
:101F08000000000000045D000001416D706C303974
:101F180000000100600042C800003F80000000008F
:101F28000000000000045D000001416D706C31305C
:101F380000000100640042C800003F80000000006B
:101F48000000000000045D000001416D706C31313B
:101F580000000100680042C800003F800000000047
:101F68000000000000045D000001416D706C31321A
:101F7800000001006C0042C800003F800000000023
:101F88000000000000045D000001416D706C3133F9
:101F980000000100700042C800003F8000000000FF
:101FA8000000000000045D000001416D706C3134D8
:101FB80000000100740042C800003F8000000000DB
:101FC8000000000000045D000001416D706C3135B7
:101FD80000000100780042C800003F8000000000B7
:101FE8000000000000045D000001416D706C313696
:101FF800000001007C0042C800003F800000000093
:102008000000000000045D000001416D706C313774
:1020180000000100800042C800003F80000000006E
:102028000000000000045D000001416D706C313853
:1020380000000100840042C800003F80000000004A
:102048000000000000045D000001416D706C313932
:1020580000000100880042C800003F800000000026
:102068000000000000045D000001416D706C32301A
:10207800000001008C0042C800003F800000000002
:102088000000000000045D000001416D706C3231F9
:1020980000000100900042C800003F8000000000DE
:1020A8000000000000045D000001416D706C3232D8
:1020B80000000100940042C800003F8000000000BA
:1020C8000000000000045D000001416D706C3233B7
:1020D80000000100980042C800003F800000000096
:1020E8000000000000045D000001416D706C323496
:1020F800000001009C0042C800003F800000000072
:102108000000000000045D000001416D706C323574
:1021180000000100A00042C800003F80000000004D
:102128000000000000045D000001416D706C323653
:1021380000000100A40042C800003F800000000029
:102148000000000000045D000001416D706C323732
:1021580000000100A80042C800003F800000000005
:102168000000000000045D000001416D706C323811
:1021780000000100AC0042C800003F8000000000E1
:102188000000000000045D000001416D706C3239F0
:1021980000000100B00042C800003F8000000000BD
:1021A8000000000000045D000001416D706C3330D8
:1021B80000000100B40042C800003F800000000099
:1021C8000000000000045D000001416D706C3331B7
:1021D80000000100B80042C800003F800000000075
:1021E8000000000000045D000001416D706C333296
:1021F80000000100BC0042C800003F800000000051
:102208000000000000045D000001416D706C333374
:1022180000000100C00042C800003F80000000002C
:102228000000000000045D000001416D706C333453
:1022380000000100C40042C800003F800000000008
:102248000000000000045D000001416D706C333532
:1022580000000100C80042C800003F8000000000E4
:102268000000000000045D000001416D706C333611
:1022780000000100CC0042C800003F8000000000C0
:102288000000000000045D000001416D706C3337F0
:1022980000000100D00042C800003F80000000009C
:1022A8000000000000045D000001416D706C3338CF
:1022B80000000100D40042C800003F800000000078
:1022C8000000000000045D000001416D706C3339AE
:1022D80000000100D80042C800003F800000000054
:1022E800000000000001340000005665746F000013
:1022F800000001003B00000000000000000000009A
:1023080000000000000000000000000000000000C5
:1023180000000000000000000000000000000000B5
:1023280000000000000000000000000002FAF08039
:10233800000100017D7840000200009896800005A9
:1023480000004C4B40000A00002625A000140000A5
:102358000F42400032000007A1200064000003D0B3
:102368009000C800000186A001F4000000C35000DE
:102378000101000061A8000201000027100005010A
:1023880000001388000A01000009C40014010000BD
:1023980003E8003201000001F4006401000000FAC3
:1023A80000C8010000006401F401000000320001CF
:0823B80002000000000000001B
:105AD000016F01030CFF1DADC111C112C1084400CB
:105AE000000000000041003800C10DC10EC10FC10F
:105AF0001044003000000000440034000000004169
:0D5B00000004FF410005FF016D00016E0073
:024219008F43D1
:10421B0075840F75A4F575A5F075A6FFE4F5A7F5E4
:10422B0084F5BA75BC9875E880F5D1F58475D10322
:10423B00F58475D48075840175D480FD7F01125F80
:10424B00C4E4FDFF12617B7BFF7A1C793890003C44
:10425B00E0FCA3E0FDA3E0FEA3E0F54C8E4B8D4A02
:10426B008C49122B47E543601B7E007FA37D007BAF
:10427B00017A007939120A7D9000397407F0A37422
:10428B0003F0801BE4F584E5EF20E11378397C0023
:10429B007D017B017A0079DC7E007FA31206E2E4CC
:1042AB00F544E544C37882965009AF441260C405C7
:1042BB004480EFE4F544AB0CAA0DA90E75F020E594
:1042CB0044A4F58285F083120721601EE54475F046
:1042DB0020A429F9EA35F0FA90000412072130E501
:1042EB0005AF441256E1054480CCE4FDFF12617B1F
:1042FB00E4F5447B007A00799312000E7C007D027A
:10430B001207E9C374079FFFE49EFEC3E5449FEECB
:10431B006480F8748098500D7BFF7A1C7940126092
:10432B0073054480CE7BFF7A1C79421260737B004D
:10433B007A0079931260737BFF7A1C794612607353
:10434B007D01E4FF12617B7BFF7A1C794A788DE655
:10435B00F54908E6F54A122B477D02E4FF12617B13
:10436B007549FF754A1D754B8C754C00754D067B59
:10437B00017A037954125CDB7B017A0379547D203B
:10438B00126149E412074E754901754A03754B5486
:09439B007BFF7A1C795C022B47C0
:105B8400E4F58420110FD211F58475D103F5BA75AB
:0D5B9400BC9875E880C374079F5407F5BBEB
:0D5BA10075420275431300D543FCD542F652
:105BAE00C2AFC2EDD2EC30EDFDD2AFAFBFEFFFAD65
:105BBE00BEED90035CCFF0A3EFF0C3E094E890034A
:0C5BCE005CE0940350047F0180027F0023
:015BDA0022A8
:104BA6001261A2C8ECC8C9EDC9CAEECACBEFCB9058
:104BB6000000E0FCA3E0FDA3E0FEA3E0240AFFE47E
:104BC6003EFEE43DFDE43CFCD31208DE5003024CFD
:104BD600941261A29000001209C17D007F00125E4E
:104BE600F58F41E54120E0352012031262097A0073
:104BF6007B647D017F011254ABE4FDFF12617B7B78
:104C0600FF7A1C796C122B477D01E4FF12617B7BD6
:104C1600FF7A1C7981122B47D2127F0122301205AE
:104C2600C212126209E54120E15C20080312620902
:104C36007A007B647D017F011254ABE4FDFF1261B3
:104C46007B7BFF7A1C7996122B477D01E4FF12616C
:104C56007B7BFF7A1C79AB122B477D03E4FF126145
:104C66007B7BFF7A1C79C0122B47E4FF125B84EF33
:104C7600600F7D017F00125EF5E4FF125B84EF702A
:104C8600F8D2087F0122300805C2081262097F00A7
:014C960022FB
:10576C007D017F00125EF57B207D057F00125C873A
:10577C00EF7027FDFF12617B7BFF7A1C79D5122B12
:10578C00477BFF7A1C79EA122B477BFF7A1C79FF47
:10579C00122B477F00125FF180F9E4900354F090D4
:1057AC000354E0FFC39405502D151215121512A8C1
:1057BC001276000876000876001512A812E4F61589
:1057CC0012A812EFF67B007D017F02123C6390035E
:0657DC0054E004F080C956
:0157E20022A4
:1060C4001512A812EFF6A812E6FFC3942A5013EF94
:1060D400C39400400D74062FF582E43400F58374F4
:0560E40001F00512228D
:056222008F397F00220E
:0F61EC00120708AB3CAA3DA93E12074E7F0122C5
:103E7A00301303126209124BA6EF60037F0022E49B
:103E8A00FDFF12617B900039E070087BFF7A1D7993
:103E9A001480627BFF7A1D7925900039E075F0075E
:103EAA00A42431F582E43423F583E493F5497401BB
:103EBA0093F54A122B47900039E075F007A4243392
:103ECA00F582E43423F583E49370087BFF7A1D7945
:103EDA00348022900039E075F007A42433F582E497
:103EEA003423F583E4937BFFB401067A1D793A8083
:103EFA00047A1D7941122B477D01E4FF12617B7B15
:103F0A00FF7A1D7948900038E0F549122B477D0366
:103F1A00E4FF12617B7BFF7A1D795D122B47300922
:103F2A000F200D0C900039E0D394004003E014F008
:103F3A00300A0F200E0C900039E0C394135003E0AE
:103F4A0004F0300B18200F15900038E0D39400408D
:103F5A000CE014F01261A29000301209C1300B3A41
:103F6A001261A2C8ECC8C9EDC9CAEECACBEFCB90A0
:103F7A000030E0FCA3E0FDA3E0FEA3E02446FFE45A
:103F8A003EFEE43DFDE43CFCD31208DE400C90000A
:103F9A0038E0D394004003E014F0300C18201015D8
:103FAA00900038E0C39464500CE004F01261A290CF
:103FBA0000341209C1300C391261A2C8ECC8C9ED2B
:103FCA00C9CAEECACBEFCB900034E0FCA3E0FDA354
:103FDA00E0FEA3E02446FFE43EFEE43DFDE43CFCB3
:103FEA00D31208DE400B900038E094645003E004DA
:103FFA00F0900005E0FF900039E06F60057F001245
:10400A0060C4900004E0FF900038E06F604C754097
:10401A0002E540C37882965041900038E0FCE412F1
:10402A0003BBE4FBFA79C878421202A7EEC0E0EFBC
:10403A00C0E0E54075F020A4AB0C250EF9E50D357E
:10404A00F0FA90000D120A27D0E0FFD0E0FE120924
:10405A0052AF401260C4054080B7900038E090002B
:10406A0004F0900039E0900005F0A209920DA20A2E
:0C407A00920EA20B920FA20C92107F007D
:014086002217
:10452400900006E06034E4F0900039E075F007A4F0
:10453400242DF9742335F0151215121512A81276CC
:10454400FF08F608C6E9C61512A812E4F61512A863
:1045540012F6FB7D047F02123C63900007E06024A6
:10456400E4F0151215121512A81276010876000847
:10457400763A1512A812F61512A812F6FB7D057FDD
:1045840002123C639003547402F0900354E0FFC39E
:10459400788296506E74062FF582E43400F583E039
:1045A4006059900354E02406F582E43400F583E472
:1045B400F0EF75F004A42434F9740035F0151215E5
:1045C400121512A812760108F608C6E9C69003541B
:1045D400E0FF24FE54071512A812F6EF24FEFFE4B0
:1045E40034FFFEEF7803CEC313CE13D8F91512A807
:1045F40012F67B007D027F02123C63900354E004B8
:10460400F080877B007A00793F7D067F0012509E00
:10461400E53F20E0047F0180027F0090003BEFF043
:1046240078DC7C007D017B017A0079397E007FA3F0
:104634001206E2E4FF125B84EF24FF92097F011269
:104644005B84EF24FF920A7F02125B84EF24FF92C3
:0E4654000B7F03125B84EF24FF920C0223C045
:0E408700E5122404F8E6FDE5122403F8E6FF36
:104095001512A812EBF61512A812EDF61512A812B4
:0440A500EFF615120B
:1040A900D2B1C2B0C2B2A812E4F6A812E6FFC39414
:1040B90004504B08E6FEC8EFC8088002C333D8FC99
:1040C9005408D394004003D38001C392B300000085
:1040D90000000000000000000000000000000000D7
:1040E90000D2B00000000000000000000000000045
:1040F90000000000000000C2B0A8120680ACA8129F
:10410900E4F6A812E6FFC39403504C0808E6FEC87B
:10411900EFC8088002C333D8FC5404D39400400389
:10412900D38001C392B3000000000000000000002A
:1041390000000000000000000000D2B000000000F4
:104149000000000000000000000000000000000066
:10415900C2B0A8120680ABA812E4F6A812E6FFC303
:104169009403504FE5122403F8E6FEC8EFC808800F
:1041790002C333D8FC5404D394004003D38001C351
:1041890092B30000000000000000000000000000E1
:10419900000000000000D2B0000000000000000094
:1041A900000000000000000000000000C2B0A812DA
:1041B9000680A8D2B2000000000000000000000044
:1041C900000000000000000000D2B0000000000064
:1041D900000000000000000000000000000000C214
:1041E900B0C2B2C2B3E5122404F8E624FF92B0D2F9
:1041F900B2C2B10000000000000000000000000091
:0942090000000000000000C2B238
:07421200E5122405F512225C
:084E4900FBE512240BF8E6FF63
:104E51001512A812EBF61512A812EDF61512A812EA
:044E6100EFF6151241
:104E65001512A812E4F67B02E5122403F8E6FDA864
:104E7500120808E6FF124095A812E4F6A812E6C348
:104E85009408504EE5122403F8E6FF5480D39400AD
:104E95004003D38001C392B300000000000000006E
:104EA500000000000000000000000000D2B000007B
:104EB50000000000000000000000000000000000ED
:104EC5000000C2B0E5122403F8EF25E0F6A81206AB
:104ED50080AAC2B3D2B200000000000000000000AA
:104EE50000000000000000000000D2B0000000003B
:104EF50000000000000000000000000000000000AD
:044F0500C2B0C2B2C2
:074F0900E5122404F5122259
:10509E00151215121512A812C6EBC608C6EAC608D6
:1050AE00C6E9C61512A812EDF61512A812EFF615DE
:0350BE00121512B6
:1050C1001512A812E4F6FB124087D2B200000000CC
:1050D10000000000000000000000000000000000CF
:1050E100D2B000000000000000000000000000003D
:1050F100000000000000C2B0C2B2A812E4F6A8127B
:10510100E6C39408503F00000000000000000000CA
:1051110000000000000000000000D2B0000000000C
:10512100000000000000000000000000000000007E
:10513100C2B008E625E0FFA2B4E4334FA81208F696
:10514100A8120680B9A81208E6FFE5122404F8CBDC
:0C515100E6CB08E6FA08E6F9EF12074E7C
:07515D00E5122407F5122200
:104F1000151215121512A812C6EBC608C6EAC60865
:104F2000C6E9C61512A812EDF61512A812EFF6156D
:034F300012151245
:104F33001512A812E4F67B01124087D2B2000000DA
:104F4300000000000000000000000000000000005E
:104F530000D2B000000000000000000000000000CC
:104F630000000000000000C2B0C2B2A812E4F6A81C
:104F730012E6C39408503F00000000000000000048
:104F83000000000000000000000000D2B00000009C
:104F9300000000000000000000000000000000000E
:104FA30000C2B008E625E0FFA2B4E4334FA812081C
:104FB300F6A8120680B9A81208E6FFE5122404F841
:0D4FC300CBE6CB08E6FA08E6F9EF12074E40
:074FD000E5122407F512228F
:0B4D7F00E4CBEFCBE512240BF8E6FFBD
:104D8A001512A812EBF61512A812EDF61512A812B2
:044D9A00EFF6151209
:104D9E001512A812E4F67B04E5122403F8E6FDA82A
:104DAE00120808E6FF124095A812E4F6A812E6C310
:104DBE009408504EE5122403F8E6FF5480D3940075
:104DCE004003D38001C392B3000000000000000036
:104DDE00000000000000000000000000D2B0000043
:104DEE0000000000000000000000000000000000B5
:104DFE000000C2B0E5122403F8EF25E0F6A8120673
:104E0E0080AAC2B3D2B20000000000000000000071
:104E1E0000000000000000000000D2B00000000002
:104E2E000000000000000000000000000000000074
:044E3E00C2B0C2B28A
:074E4200E5122404F5122221
:104FD700151215121512A812C6EBC608C6EAC6089E
:104FE700C6E9C61512A812EDF61512A812EFF615A6
:034FF7001215127E
:104FFA001512A812E4F67B03124087D2B200000011
:10500A000000000000000000000000000000000096
:10501A0000D2B00000000000000000000000000004
:10502A0000000000000000C2B0C2B2A812E4F6A854
:10503A0012E6C39408503F00000000000000000080
:10504A000000000000000000000000D2B0000000D4
:10505A000000000000000000000000000000000046
:10506A0000C2B008E625E0FFA2B4E4334FA8120854
:10507A00F6A8120680B9A81208E6FFE5122404F879
:0D508A00CBE6CB08E6FA08E6F9EF12074E78
:07509700E5122407F51222C7
:0E49B7001512A812EDF61512A812EFF6151241
:1049C5001512A812E4F67B06E5122403F8E6FDA805
:1049D500120808E6FF124095D2B30000000000005F
:1049E5000000000000000000000000000000D2B040
:1049F50000000000000000000000000000000000B2
:104A050000000000C2B0D2B30000000000000000AA
:104A1500000000000000000000000000D2B000000F
:104A25000000000000000000000000000000000081
:104A35000000C2B0C2B3000000000000000000008A
:104A450000000000000000000000D2B000000000DF
:104A55000000000000000000000000000000000051
:104A6500C2B0A812E4F6A812E6C394065031C2B348
:104A75000000000000000000000000000000000031
:104A850000000000D2B0000000000000000000009F
:104A950000000000000000000000C2B00680C72032
:084AA500B4047F0180027F00D0
:074AAD00051205120512229B
:1043A400151215121512A812C6EBC608C6EAC608DD
:1043B400C6E9C61512A812EDF61512A812EFF615E5
:0543C400121512151294
:1043C9001512A812E4F67B06E5122405F8E6FDE5C8
:1043D900122404F8E6FF124095D2B3000000000051
:1043E900000000000000000000000000000000D2F2
:1043F900B000000000000000000000000000000004
:104409000000000000C2B0D2B300000000000000AC
:1044190000000000000000000000000000D2B00011
:104429000000000000000000000000000000000083
:10443900000000C2B0C2B30000000000000000008C
:104449000000000000000000000000D2B0000000E1
:104459000000000000000000000000000000000053
:1044690000C2B0A812E4F6A812E6C394065031C2FD
:10447900B300000000000000000000000000000080
:104489000000000000D2B0000000000000000000A1
:104499000000000000000000000000C2B00680C754
:1044A900A812E4F6A812E6C39410504E00000000CA
:1044B90000000000000000000000000000000000F3
:1044C900D2B0000000000000000000000000000061
:1044D900000000000000C2B008C9E8C909E725E0EA
:1044E900FF19E733FEA2B4E433FDEF4DFFA812082C
:1044F900EEF608EFF6A8120680AAA81208C9E8C9BC
:10450900E7FFE5122405F8CBE6CB08E6FA08E6F959
:04451900EF12074E48
:07451D00E5122408F512224B
:105C87001512A812EBF61512A812EDF61512A812A6
:045C9700EFF61512FD
:105C9B00A8120808E6FDA81208E6FF1249B7EF7034
:105CAB0003FF80257B00A9127A00A8120808E6FDE5
:105CBB00A81208E6FF1243A4E5122403F9A812E682
:095CCB006770047F0180027F0074
:075CD400E5122404F5122281
:10353B001512A812EBF61512A812EDF61512A81219
:08354B00EFF6E51224FBF51276
:103553001512A812E4F67B06E5122407F8E6FDE54A
:10356300122406F8E6FF124095D2B30000000000D3
:10357300000000000000000000000000000000D276
:10358300B000000000000000000000000000000088
:103593000000000000C2B0C2B30000000000000041
:1035A30000000000000000000000000000D2B00096
:1035B3000000000000000000000000000000000008
:1035C300000000C2B0C2B300000000000000000011
:1035D3000000000000000000000000D2B000000066
:1035E30000000000000000000000000000000000D8
:1035F30000C2B0A812E4F6A812E6C394065031D272
:10360300B300000000000000000000000000000004
:103613000000000000D2B000000000000000000025
:103623000000000000000000000000C2B00680C7D8
:10363300D2B2000000000000000000000000000003
:10364300000000000000C2B2D2B30000000000007E
:103653000000000000000000000000000000D2B0E5
:103663000000000000000000000000000000000057
:1036730000000000C2B0C2B3000000000000000060
:10368300000000000000000000000000D2B00000B5
:103693000000000000000000000000000000000027
:1036A3000000C2B0D2B30000000000000000000020
:1036B30000000000000000000000D2B00000000085
:1036C30000000000000000000000000000000000F7
:1036D300C2B0A812E4F6A812E6C394065031C2B3EE
:1036E30000000000000000000000000000000000D7
:1036F30000000000D2B00000000000000000000045
:1037030000000000000000000000C2B00680C7A84F
:1037130012E4F6A812E6C39410504EE5122407F8FB
:10372300E6FF5480D394004003D38001C392B300D7
:103733000000000000000000000000000000000086
:10374300000000D2B00000000000000000000000F4
:10375300000000000000000000C2B0E5122407F8DA
:10376300EF25E0F6A8120680AAD2B20000000000FE
:10377300000000000000000000000000000000C284
:10378300B2A81208E4F608F6A81208C9E8C9C309E2
:0C379300E7941019E79427504420B4413B
:10379F00E5122403F87601E5122403F8E6D394002A
:1037AF004023E5122404F87613E5122404F8E6D337
:1037BF009400400900E5122404F81680ECE5122469
:0537CF0003F81680D292
:0C37D400A812080806E61870AE0680ABCC
:0737E000E5122408F5122296
:0E5EF5001512A812EDF61512A812EFF61512EE
:105F0300A8120808E6600C7B047D01A81208E6FFCE
:105F1300124D8A7B00A9127A007D01A81208E6FFC0
:075F2300124FD7A812E6FFA0
:075F2A000512051205122209
:103A3500A912151215121512A8127600087600089B
:103A4500C6E9C6E5122410F8E61512A812F6E51225
:103A55002410F8E61512A812F6E5122410F8E6FB74
:043A65007D027F025D
:103A69001512A812EBF61512A812EDF61512A812E6
:083A7900EFF6E51224F9F51245
:103A81002408F8E664026003023C5AE512240CF8AB
:103A9100CBE6CB08E6FA08E6F9120902A8121209E8
:103AA100B5E5122407F8E6B4020F7F007EFF7D7FA3
:103AB1007C47A812120978804EE5122407F8E6B473
:103AC100821FE4FBFA79207840E8C0E0A8121209CD
:103AD1006CD0E0F81202A77B007AFF797F784780EB
:103AE10026E5122407F8E6B4832DE4FBFA79C878B9
:103AF10041E8C0E0A81212096CD0E0F81202A77BDD
:103B0100007AFF797F784712019E1203EFE51224B4
:103B110004F8EEF608EFF61512A812E4F67B05E5B7
:103B210012240BF8E6FDE512240AF8E6FF1240958F
:103B3100E5122406F8E4F6E5122406F8E6FFC3943C
:103B410004503FEF94014003D38001C392B30000BE
:103B51000000000000000000000000000000000064
:103B61000000D2B0000000000000000000000000D2
:103B71000000000000000000C2B0E5122406F806B3
:103B810080B5E5122406F8E4F6E5122406F8E6C34A
:103B910094045051E512240BF8E6FF5408D3940025
:103BA1004003D38001C392B3000000000000000075
:103BB100000000000000000000000000D2B0000082
:103BC10000000000000000000000000000000000F4
:103BD1000000C2B0E512240BF8EF25E0F6E512244F
:103BE10006F80680A4E5122406F8E4F6E512240698
:103BF100F8E6C394105060E5122404F8E6FE08E6E6
:103C0100FFEE5480FCD3E49400EC94004003D38095
:103C110001C392B30000000000000000000000009A
:103C21000000000000000000D2B000000000000011
:103C31000000000000000000000000000000C2B011
:103C4100E5122404F8EF25E0FFEE33F608EFF6E580
:0B3C5100122406F8068095D2B17F0116
:073C5C00E512240FF512220E
:103C63001512A812EBF61512A812EDF61512A812EA
:083C7300EFF6E51224F7F5124B
:103C7B00E512240AF8E66401705FE512240CF8E6FD
:103C8B00FD245EF582E43403F583E4F0124E49A87B
:103C9B00121209CD00000000123A357B00E5122408
:103CAB0004F97A007D00E512240BF8E6FF124FD7DA
:103CBB00E5122404F8C9E8C9E512240CF8E6FF74F0
:103CCB0001C8EFC8088002C333D8FC47F7E51224BC
:103CDB0004F8E6FB7D00124D83E512240AF8E66436
:103CEB00026003023D7CE512240EF8CBE6CB08E61E
:103CFB00FA08E6F9120902A8121209B5123A35E4CC
:103D0B00FFFEFDFCA8121209781203447029E5127C
:103D1B00240CF8E6245EF582E43403F583E0FFE53A
:103D2B0012240DF8E6FE7401C8EEC8088002C333F6
:103D3B00D8FCF45FF08026E512240CF8E6245EF53F
:103D4B0082E43403F583E0FFE512240DF8E6FE74FC
:103D5B0001C8EEC8088002C333D8FC4FF0E512242B
:103D6B000CF8E6FD245EF582E43403F583E0124E95
:103D7B0049E512240AF8E664046003023E36E512B4
:103D8B00240EF8CBE6CB08E6FA08E6F9120902E5B1
:103D9B00122405F81209B5E5122405F812096C7DF9
:103DAB0003124D7FE5122405F8E8C0E012096C7888
:103DBB00081208EFD0E0F81209B5E5122405F81245
:103DCB00096C7D04124D7FE5122405F8E8C0E01262
:103DDB00096C78081208EFD0E0F81209B5E5122447
:103DEB0005F812096CE4CBEFCB7D05124D83E51280
:103DFB002405F8E8C0E012096C78081208EFD0E04F
:103E0B00F81209B5E5122405F812096CE4CBEFCBD7
:103E1B007D06124D83E5122405F8E8C0E012096C0B
:103E2B0078081208EFD0E0F81209B5E512240AF869
:103E3B00E664057031E512240EF8CBE6CB08E6FA02
:103E4B0008E6F9120708FFE5122404F8EFF6D394FD
:103E5B00144007E5122404F87614E5122404F8E65E
:083E6B00FB7D02124D837F0173
:073E7300E5122411F51222F3
:10601D0020202020557067726164696E6700202012
:10602D0020204669726D776172652E2E2E002452E6
:0B603D0065763A20343931362024000B
:0F5B0D000184FF420189FFFF44018B000000006B
:102F5400E47880F61261C8C28575840F75E104E4D3
:102F6400F5E275E344F58475B7B075840F758A830B
:102F7400F597438901758D01758F01758E04F541AF
:102F8400F5420542E54270020541640F454170F285
:102F9400438902E4F541F542AE41AF42E4FCFD7BD6
:102FA400507AC3F9F8D31208C8400FE58920E40A1F
:102FB4000542E54270E2054180DE7597021257E34F
:102FC40012610BE4FF12612A43EF04E4F541F54278
:102FD4007D01AF42125FC40542E54270020541C360
:102FE4009402E541940040E8E4F520C229C227C2D6
:102FF4002DC22CC22B7880F608F67886F618F6785F
:103004008BF6F541F542748F2542F582E43401F5DF
:1030140083E4F00542E54270020541B400E8E5416D
:10302400B401E3E4F541F542748F2542F582E434BA
:1030340002F583E4F00542E542700205416440452F
:103044004170E5E4F584E5EF20E10CE5EF5408D3A5
:1030540094004003D38001C392037D08E4FF125D12
:103064007E7D087F01125D7E12576CE4788AF678C3
:1030740082F6AB0CAA0DA90E7882E6FF75F020A4A7
:10308400F58285F083120721FE788A26F6EE600524
:1030940078820680DDEFD394004030AB0CAA0DA9F2
:1030A4000E90000D120A27120708FF745512074EDE
:1030B40012070864556002D22B74AA12074E120735
:1030C4000864AA6002D22BEF12074EE4F584E5EF00
:1030D4005402D3940040047F018002E4FF124C9711
:1030E4008F40E54020E036C22874FF788DF608F65C
:1030F40008F608F67E007F107D007B007A00799345
:10310400120A7D7549FF754A1D754B71754C007522
:103114004D107B007A007993125CDB8002D22890F8
:103124006042E493FF3395E0FEEF24D0FFEE34FFDA
:10313400FE7C007D64120782AA06AB07906041E41E
:1031440093FF3395E0FEEF24D0FFEE34FFFE7C03C3
:103154007DE8120782EF2BFBEE3AFA906043E4938A
:10316400FF3395E0FEEF24D0FFEE34FFFE7C007DBC
:103174000A120782EF2BFFEE3AFEA3E493FD339588
:10318400E0FCED24D0FDEC34FFCD2F7892F6ED3E3B
:1031940018F6E54030E103023241E4F541F542E539
:1031A40042AE417805C333CE33CED8F9FFAB0CAA77
:1031B4000DA90EF5828E831207216078E92FF9EAB2
:1031C4003EFA90000412072120E25EE4F53FE53F59
:1031D400C3786F965053E542AE417805C333CE337E
:1031E400CED8F9AB0CAA0DA90EF5828E8312072155
:1031F400FF7E00C006C0077D00E542AE417805C3EE
:1032040033CE33CED8F929F9EA3EFA90000D120AEA
:1032140027788AE6853FF0A429F9EA35F0FAD00741
:10322400D006120A7D053F80A50542E542700205DD
:10323400410231A37F01124219C22A8007E4FF121E
:103244004219D22AE4F541F5427A007B967D03AF18
:10325400421254AB0542E54270020541C39402E5B3
:0532640041940040E46C
:013269002242
:05622700788BE6FF2268
:0300230002478D04
:10478D00C0E0C0F0C083C082C0D075D000C000C0F2
:10479D0001C002C003C004C005C006C00730993E69
:1047AD00C2997886067986E77881667015F67886DF
:0147BD00F605
:0D47BE0075270A75281300D528FCD527F6AD
:0447CB00C285801C07
:0D47CF0075271475281300D528FCD527F692
:1047DC007886E6248FF582E43402F583E0F599209F
:1047EC009803024888209A08202905C29802488418
:1047FC00C29A7885E606248FF582E43401F583E5C8
:10480C0099F0C298E6FFB4011290018FE0FE70039C
:10481C00F68069EE54072402788CF6EFB4020D781A
:10482C008CE6B40907900190E02403F67885E6FF46
:10483C00B40007E4B40103F68042EFC3788C9640D1
:10484C003B7885E624FFFDE434FFFC7B017A01799B
:10485C008F1255C97885E6248EF582E43401F583F0
:08486C00E06F60047600801487
:0D48740075271475281300D528FCD527F6EC
:10488100120B4378857600D007D006D005D004D02E
:1048910003D002D001D000D0D0D082D083D0F0D0CC
:0248A100E03203
:10002600900190E075F020A4AB0C250EF9E50D3596
:10003600F0FA90000D120A27788BE6FF18E68FF08B
:10004600A4252BF582E435F0F583120721FF7B000A
:040056007A0079298A
:10005A008F398B3A8A3B893CE4F584EA494B601C28
:10006A00AB3AAA3BA93C120708FFE539FD7C00120E
:0C007A006216AB3AAA3BA93CEF12074EFD
:0D008600753D14753E1300D53EFCD53DF6CA
:0E0093008539997F01125FF13099FDC29922E3
:105F310090028F7478F07885E6248EF582E434013E
:095F4100F583E0900290F07F026C
:095F4A00E4F5847881EFF6D285BC
:0D5F5300753914753A1300D53AFCD539F6AE
:075F600090028FE0F5992289
:105E6600C9EFC9E964017028EDC39B4034786FE639
:105E7600FFEB2FFFE433FEEDC39FEE6480F87480E2
:105E860098501ED229C3ED9B788BF678877601222F
:105E9600B90214ED6B700AD229788BF678877602F0
:085EA60022C229E47887F622EC
:105A6F00C9EFC9BAFF15BBFF12ED6B7002EC6A707C
:105A7F0049D229788BF67887E9F622E964017025F7
:105A8F00C3ED9BEC9A401C786FE62BFFE43AFEC304
:105A9F00ED9FEC9E500DD229C3ED9B788BF6788746
:105AAF007601228015B90218ED6B7002EC6A700A4C
:105ABF00D229788BF67887760222C229E47887F686
:015ACF0022B4
:100B430090018FE0FF54F8F52AE4F584EF120A5779
:100B53000B90090B9D0A0BB0100BB9110BCA120BAA
:100B6300E1190BF71A0C1C200C25280CA6290DA83B
:100B7300330DE3370E12390E2C410E37490E415017
:100B83000E89610D72700E819800000EB99001906C
:100B9300E0FD788EE6FB7F018027900190E0FCA3C7
:100BA300E0FD788DE6FA08E6FB7F01802BD22978F9
:100BB300877603020EB9900190E0FD7890E6FB7F03
:100BC30002125E66020EB9900190E0FCA3E0FD788C
:100BD3008FE6FA08E6FB7F02125A6F020EB9900104
:100BE30090E0FD788EE6FB7F01125E66202903020A
:100BF3000EB9801A900190E0FCA3E0FD788DE6FA2F
:100C030008E6FB7F01125A6F202903020EB99002F6
:100C13008F7478F07F01020EB6E4F58475EF10024D
:100C23000EB9C2ACE4F529D285FB7A0079297F7F1E
:100C330012005A7B007A0079297F1812005A7B0030
:100C43007A0079297F0512005A7882E612005378D8
:100C53008DE6120053788EE6120053788FE6120069
:100C6300537890E61200537891E61200537892E697
:100C7300120053E4F52B7493252BF8E61200530569
:100C83002BE52BC3941040EE7B007A007900AF294B
:030C930012005AF2
:0D0C960075370A75381300D538FCD537F6D0
:100CA300020D5D900190E0FFC37882964003020D30
:100CB30064EF75F020A4250EF9E50D35F0850C34AD
:100CC300F5358936C2ACE4F529D285FB7A0079295A
:100CD3007F7F12005A7B007A0079297F0D12005A18
:100CE300AB34AA35A936120708120053AB34AA3520
:100CF300A936900001120050AB34AA35A9369000F2
:100D030002120050AB34AA35A936900003120050EA
:100D1300AB34AA35A936900004120050E4F52BAB8E
:100D230034E5362405F9E43535FA7E00E9252BF957
:100D3300EE3AFA120708120053052BE52BC3940869
:0D0D430040DD7B007A007900AF2912005AD4
:0D0D500075370A75381300D538FCD537F615
:100D5D00C285D2AC020EB990028F7478F0E4A3F084
:100D6D007F02020EB61261B578131209B590028F8B
:100D7D00747CF07813E6A3F008E6A3F008E6A3F080
:100D8D0008E6A3F07C007D057B017A02798F125570
:100D9D00C9900294EFF07F06020EB6900190E0FF2D
:100DAD00B4010FA3E0FDA3E0788DCDF608EDF602BA
:100DBD000E81EFB4020A900191E0788DF6020E815A
:100DCD00900190E0B4030CA3E0FFA3E0788FCFF681
:100DDD0008EFF6020E81E4F52B900190E0FFE52B74
:100DED00C39F501B7491252BF582E43401F583E0EC
:100DFD00FF7493252BF8EFF6052BE52BB410DAE4F1
:100E0D0078A2F6806F7A007B327D01788BE6FF1237
:100E1D0054AB900190E0FDE4FF125D7E020EB9909F
:100E2D000190E024FF9202020EB9900190E024FFA0
:100E3D0092018078788BE66005752D02800B202C51
:100E4D0005752D038003752D0190028F7479F0A324
:100E5D00E52DF07C007D027B017A02798F1255C958
:100E6D00900291EFF07F03125F4AE52D6401703C13
:100E7D00D22D8002D227788076F180307A007B32B5
:100E8D007D017F001254AB90028F7479F090019028
:100E9D00E0900290F07C007D027B017A02798F1246
:100EAD0055C9900291EFF07F03125F4AE52A64A0C5
:100EBD0060030210C890018FE064A16003020FB8B7
:100ECD00A3E0C37882964003020FADAB0CAA0DA927
:100EDD000EE0FF75F020A4F58285F083120721F551
:100EED002DEF75F020A429F9EA35F0FA90000412DF
:100EFD00072130E237900190E01262228F2D90028F
:100F0D008F747FF0A3E52DF02402FDE433FC7B010B
:100F1D007A02798F1255C97491252DF582E4340228
:100F2D00F583EFF0E52D2403FF0210C5900190E04D
:100F3D00FF126222C2ACE4F529D285E52DD39406C9
:100F4D00402B7B007A0079297F7F12005A7B007A33
:100F5D00007929AF2D12005AE4F52BE52BC3952D01
:100F6D005007120026052B80F2052D8018E52D2443
:100F7D0078120053E4F52BE52BC3952D5007120085
:100F8D0026052B80F27B007A007900AF2912005ADA
:0D0F9D0075370A75381300D538FCD537F6C6
:100FAA000210B790028F7478F07F010210C5900189
:100FBA008FE064A260030210C87882E6FFA3E0FE15
:100FCA00C39F40030210BDA3E0FDC39F400302106C
:100FDA00BDEE9D40030210BD900190E0F52BE4F5B3
:100FEA0032F533900191E0FFE52BD39F5026AF2BCA
:100FFA00126222AB0CAA0DA90E75F020E52BA4F5FE
:10100A008285F0831207212533F533E43532F53230
:10101A00052B80CFC2ACE4F529D285FB7A00792969
:10102A007F7F12005AC3E5339480E5329400500260
:10103A008007E5324480120053AF33120054900106
:10104A0090E0F52B900191E0FFE52BD39F5046E409
:10105A00F52CAB0CAA0DA90E75F020E52BA4F58290
:10106A0085F083120721FFE52CC39F5024E52B75D9
:10107A00F020A429F9EA35F0FA90000D120A27782F
:10108A008BE6FF18E68FF0A4252C120049052C8068
:10109A00C1052B80AF7B007A007900AF2912005A74
:0D10AA0075370A75381300D538FCD537F6B8
:1010B700C285D2AC800B90028F7478F07F01125FEB
:1010C7004AE52A6458704DFA7B327D01788BE6FF3A
:1010D7001254AB753C01753D02753E907B017A0158
:1010E70079901261EC8F2DE52D247890028FF0EF27
:1010F7002401FDE433FC7B017A02798F1255C97410
:1011070090252DF582E43402F583EFF0E52D2402D6
:10111700FF125F4AE52A64806009E52A6488600354
:101127000212ED7887E6B4010F7A007B327D0178F1
:101137008BE6FF1254AB801AE4F52BE52BC3786FCF
:1011470096500F7A007B327D01AF2B1254AB052BE3
:1011570080E990018FE05407F52DB4070A752C013B
:10116700A3E0F52DA38006E4F52C900190E0F52E81
:10117700152DE52EC378829640030212DAAB0CAA2E
:101187000DA90E75F020E52EA4F58285F0831207D0
:1011970021FFE52DD39F40028F2D7887E6B4010903
:1011A700788BE6F531F5308009E4F530786FE61491
:1011B700F531788BA630788BE6D395314003021250
:1011C700B1E4F52BE52BC3952D40030212A6E52EBE
:1011D70075F020A4AB0C250EF9E50D35F0FA90005B
:1011E7000412072130E2030212A190000112072125
:1011F70064387041E52DD394044011E52C252B2448
:1012070091F582E43401F583E0FD80707885E6C3CB
:10121700952BFFE49400FE748D2FF58274013EF543
:1012270083E0FDE52E75F020A4AB0C250EF9E50D46
:1012370035F0FA8047AB0CAA0DA90E75F020E52E04
:10124700A4F58285F083120721FF7885E6C39FFF07
:10125700E49400FE7C00EF252BFFEC3EFEEF252CEF
:10126700FFEC3EFE748E2FF58274013EF583E0FDA0
:10127700E52E75F020A429F9EA35F0FA90000D1251
:101287000A27788BE6FF18E68FF0A4FFE52B2FF5EA
:1012970082E435F0F583ED120760052B0211CBAF21
:1012A7002E1260C4788B060211BD788BA630E52E0E
:1012B70075F020A4AB0C250EF9E50D35F0FA90007A
:1012C7000412072130E5047884A62EE52A64887085
:1012D700158010E52EB4FF0E900191E0F520E52A68
:1012E700B48803125F31E52A64A8600302142578E5
:1012F70087E6B4010F7A007B327D01788BE6FF1217
:1013070054AB801AE4F52BE52BC3786F96500F7A10
:10131700007B327D01AF2B1254AB052B80E9900186
:1013270090E030E711547FFEA3E0FDEEF532EDF5D6
:1013370033752C03800C900190E0753200F53375FE
:101347002C02748F252CF582E43401F583E0FF74B9
:1013570090252CF582E43401F583E0F52F8F2EE5F7
:101367002ED3952F4003021422E52EC37882964090
:101377000302141DAB0CAA0DA90E75F020E52EA4CF
:10138700F58285F083120721F52D7887E6B40109E8
:10139700788BE6F531F5308009E4F530786FE6149F
:1013A700F531788BA630788BE6D39531505EE4F52E
:1013B7002BE52BC3952D504AE52E75F020A4AB0CD9
:1013C700250EF9E50D35F0FA90000412072120E209
:1013D7002DE52C252B2491F582E43401F583E0FDDE
:1013E70090000D120A27788BE6FF18E68FF0A4FF0E
:1013F700E52B2FF582E435F0F583ED120760052B19
:1014070080AFAF2E1260C4788B06809A788BA63097
:0E141700E52D252CF52C052E021366125F31F3
:0114250022A4
:095BDB0090001D12084AFFAEF013
:105BE4008E478F48900189E065477004A3E06548BB
:105BF400603A90017F740AF0E547A3F0E548A3F00A
:105C04007C007D037B017A01797F1255C990018262
:105C1400EFF07B017A01797F754E017D047C0012DF
:0D5C24005419900189E547F0A3E548F022EE
:035D2D00CCEECCED
:105D300090017F741AF0A3ECF0EFA3F07C007D03D8
:105D40007B017A01797F1255C9900182EFF07B01C6
:105D50007A01797F754E017D047C001254197B0114
:105D60007A01797F7D0A7C00125164EF7002FF2274
:0D5D700090017FE0647860037F00227F01D6
:015D7D002203
:105F97007A007B327D017F011254AB74FF90018937
:105FA700F0A3F07F0A90017FE4F0A3DFFC7B017A86
:0D5FB70001797F754E017D0A7C00025419AE
:10466200E4F53FE53FC3788296400302478CE53F7D
:1046720075F020A4AB0C250EF9E50D35F0FA90008B
:104682000412072120E403024787125BDB90017FBB
:1046920074A1F0E53F75F020A4AB0C250EF9E50DF1
:1046A20035F0FA90001F120721900180F07C007D06
:1046B200027B017A01797F1255C9900181EFF07B6B
:1046C200017A01797FE4F54E7D03FC1254197B01D6
:1046D2007A01797F7D647C001251648F40E540C38A
:1046E20094025002804DE5402476FF90017FE06FF6
:1046F2006002803FAB0CAA0DA90E75F020E53FA425
:10470200F58285F083120721FFE54024FE6F6002E7
:104712008021E54024FFFDE434FFFC7B017A01792E
:104722007F1255C9747E2540F582E43401F583E099
:104732006F6007AF3F125F97804BC2AFAB0CAA0D01
:10474200A90E75F020E53FA4F58285F083120721BA
:10475200FF7E00EEC0E0EFC0E0E53F75F020A42947
:10476200F9EA35F0FA90000D120A27C8E9C8CCEA36
:10477200CCCDEBCD7B017A017980D0E0FFD0E0FE99
:0A4782001206E2D2AF053F024665C1
:01478C00220A
:0256E1008F45F3
:1056E300EF75F020A4AB0C250EF9E50D35F0FA1299
:1056F3005BDBAB0CAA0DA90E75F020E545A4F58282
:1057030085F083120721F546248190017FF0E5455A
:1057130075F020A429F9EA35F0FA90001F12072149
:10572300900180F0AF467E0090000D120A27788129
:105733007C017D011206E2E5462402FDE433FC7B95
:10574300017A01797F1255C974812546F582E434C3
:1057530001F583EFF07B017A01797FE5462403FDB0
:09576300E433FCE4F54E02541994
:105E1D001261A2C8ECC8C9EDC9CAEECACBEFCB90CE
:105E2D00018BE0FCA3E0FDA3E0FEA3E0240AFFE468
:105E3D003EFEE43DFDE43CFCD31208DE400C124670
:105E4D00621261A290018B1209C17884E6FFF460A1
:095E5D00071256E1788476FF2259
:10F000007880E664F1600302F60CE4F544F5457897
:04F0100081E6601F16
:0DF01400754A0A754B1300D54BFCD54AF622
:10F021000545E5457002054464107004E544642714
:10F0310070DCC2AF7584015398FC75FFDE75FFADBE
:10F04100E4F540F53FE4F58420982EE4F544F545D8
:0EF05100209822C3E5459488E5449413501797
:0DF05F00754A0A754B1300D54BFCD54AF6D7
:10F06C000545E54570DF054480DBB28680CF859988
:10F07C003FC298E53F641A600302F14CF544F54534
:0EF08C00209822C3E5459488E544941350175C
:0DF09A00754A0A754B1300D54BFCD54AF69C
:10F0A7000545E54570DF054480DB3098928599403A
:10F0B700C298E4F544F545209822C3E5459488E5D0
:05F0C7004494135017F2
:0DF0CC00754A0A754B1300D54BFCD54AF66A
:10F0D9000545E54570DF054480DB20980302F046CD
:10F0E900859940C298E4F544F545209822C3E54541
:08F0F9009488E54494135017BC
:0DF10100754A0A754B1300D54BFCD54AF634
:10F10E000545E54570DF054480DB20980302F04697
:09F11E00859940C298D285C2997E
:0DF12700754A14754B1300D54BFCD54AF604
:06F134007599783099FD89
:0DF13A00754A0A754B1300D54BFCD54AF6FB
:10F14700C28502F5FEE53F6450600302F1DCF54439
:10F15700F545209822C3E5459488E5449413501754
:0DF16700754A0A754B1300D54BFCD54AF6CE
:10F174000545E54570DF054480DB20980302F04631
:09F18400859940C298D285C29918
:0DF18D00754A14754B1300D54BFCD54AF69E
:08F19A007599793099FDC299C5
:0DF1A200754A14754B1300D54BFCD54AF689
:08F1AF007599013099FDC29928
:0DF1B700754A14754B1300D54BFCD54AF674
:06F1C400E4F5993099FD0D
:0DF1CA00754A0A754B1300D54BFCD54AF66B
:0FF1D700C28502F5FEE53F6401703ED285C29904
:0DF1E600754A14754B1300D54BFCD54AF645
:08F1F3007599783099FDC2996D
:0DF1FB00754A14754B1300D54BFCD54AF630
:06F20800E4F5993099FDC8
:0DF20E00754A0A754B1300D54BFCD54AF626
:10F21B00C28502F5FEE53F6402600302F2E2F544AB
:10F22B00F545209822C3E5459488E544941350177F
:0DF23B00754A0A754B1300D54BFCD54AF6F9
:10F248000545E54570DF054480DB20980302F0465C
:10F25800859940C298E4F541E54013B39286E540AC
:10F2680025E0FEC3E49400EE94F0502AE5407F00C8
:10F2780025E0FEC394E0501EE54020E01FE4F5843D
:10F2880043B701758F038E468F478F828E83F05365
:10F29800B7F0F58F80037541FFE4F584D285C299F4
:0DF2A800754A14754B1300D54BFCD54AF682
:08F2B5007599783099FDC299AA
:0DF2BD00754A14754B1300D54BFCD54AF66D
:06F2CA008541993099FD19
:0DF2D000754A0A754B1300D54BFCD54AF664
:10F2DD00C28502F5FEE53F6403600302F42DF5449B
:10F2ED00F545209822C3E5459488E54494135017BD
:0DF2FD00754A0A754B1300D54BFCD54AF637
:10F30A000545E54570DF054480DB20980302F04699
:10F31A00859940C298E4F544F545209822C3E5450D
:08F32A009488E5449413501788
:0DF33200754A0A754B1300D54BFCD54AF601
:10F33F000545E54570DF054480DB20980302F04664
:10F34F00859942C298E540139286E54025E0FEC3B9
:10F35F00E49400EE94F0400302F046E5407D002572
:10F36F00E0FCC394E0400302F046E4F58443B701A8
:10F37F00758F01E54275F020A42DFFE5F03CF546B1
:10F38F008F47E4F584F543E543C394205048E4F5F3
:10F39F0044F545209822C3E5459488E544941350DD
:01F3AF001746
:0DF3B000754A0A754B1300D54BFCD54AF683
:10F3BD000545E54570DF054480DB20980302F046E6
:10F3CD000547E547AE467002054614F5828E83E586
:10F3DD0099F0C298054380B1E4F58453B7F0F58FE9
:06F3ED00F584D285C299EF
:0DF3F300754A14754B1300D54BFCD54AF636
:08F400007599783099FDC2995D
:0DF40800754A14754B1300D54BFCD54AF620
:06F41500E4F5993099FDB9
:0DF41B00754A0A754B1300D54BFCD54AF617
:10F42800C28502F5FEE53F6404600302F4DDF5449D
:10F43800F545209822C3E5459488E5449413501770
:0DF44800754A0A754B1300D54BFCD54AF6EA
:10F455000545E54570DF054480DB20980302F0464D
:10F46500859940C298E54025E0F548754900E4F5E1
:10F4750041F544F5450549E549AE4870020548148E
:10F48500F5828E83E4932541F5410545E5457002F6
:0EF4950005447004E544640270DBD285C29920
:0DF4A300754A14754B1300D54BFCD54AF685
:08F4B0007599783099FDC299AD
:0DF4B800754A14754B1300D54BFCD54AF670
:06F4C5008541993099FD1C
:0DF4CB00754A0A754B1300D54BFCD54AF667
:10F4D800C28502F5FEE53F6405600302F5F3F544D5
:10F4E800F545209822C3E5459488E54494135017C0
:0DF4F800754A0A754B1300D54BFCD54AF63A
:10F505000545E54570DF054480DB20980302F0469C
:10F51500859940C298E4F544F545209822C3E54510
:08F525009488E544941350178B
:0DF52D00754A0A754B1300D54BFCD54AF604
:10F53A000545E54570DF054480DB20980302F04667
:09F54A00859942C298D285C2994C
:0DF55300754A14754B1300D54BFCD54AF6D4
:08F5600075997F3099FDC299F5
:0DF56800754A14754B1300D54BFCD54AF6BF
:10F575007599203099FDE54025E0FCE54275F020C0
:10F58500A42400FFE5F03CF5488F49E4F541F54337
:02F59500C29919
:0DF59700754A14754B1300D54BFCD54AF690
:10F5A400854982854883E493F5993099FD0549E5B9
:10F5B40049AE487002054814F5828E83E4932541D0
:0BF5C400F5410543E543B420C8C2999F
:0DF5CF00754A14754B1300D54BFCD54AF658
:06F5DC008541993099FD04
:0DF5E200754A0A754B1300D54BFCD54AF64F
:10F5EF00C285800BE53FB40606E4F58475EF10E5A0
:0DF5FF003F6407600302F0467880F6D2AF4B
:01F60C0022DB
:10553C007F00125FF120280B7A007B327D017F0007
:10554C001254AB302B0B7A007B1E7D017F00125462
:10555C00AB302717302C147A007B327D01788BE628
:10556C00FF1254ABC2271252DBD228202A0C302C4B
:10557C0009788076F11252DBD22A302D2A302C2772
:10558C00C22D126209E4FDFF12617B7BFF7A607908
:10559C001D1260737D01E4FF12617B7BFF7A6079E1
:1055AC002B12607312F000202C121261A2E47B2CDF
:0D55BC007A01F9F8C31208DE5002D22C2249
:0E61FB00122F5412553C125E1D12452480F5E1
:1048A300005EBCE2613FDD83C29C7E20A3FD1F410D
:1048B3009DC3217FFCA2401E5F01E3BD3E6082DCFD
:1048C300237D9FC1421CFEA0E1BF5D0380DE3C62ED
:1048D300BEE0025CDF81633D7C22C09E1D43A1FFDD
:1048E3004618FAA427799BC584DA3866E5BB5907CD
:1048F300DB856739BAE406581947A5FB7826C49ABD
:10490300653BD987045AB8E6A7F91B45C6987A24AC
:10491300F8A6441A99C7257B3A6486D85B05E7B99C
:104923008CD2306EEDB3510F4E10F2AC2F7193CD8C
:10493300114FADF3702ECC92D38D6F31B2EC0E507C
:10494300AFF1134DCE90722C6D33D18F0C52B0EE6C
:10495300326C8ED0530DEFB1F0AE4C1291CF2D735C
:10496300CA947628ABF517490856B4EA6937D58B4C
:104973005709EBB536688AD495CB2977F4AA48163C
:10498300E9B7550B88D6346A2B7597C94A14F6A82C
:10499300742AC896154BA9F7B6E80A54D7896B351C
:1049A300000000002B6096CBDDEE002C96CBDDE5FE
:0449B300EEF7FAFD24
:055B1C00C1B0016A0A9E
:10618F0074FFF50BF50AF509F508AF0BAE0AAD096B
:02619F00AC084A
:0161A10022DB
:1055C90015121512A812ECF608EDF615121512159A
:1055D90012A812C6EBC608C6EAC608C6E9C6E5128D
:0455E90024FCF51297
:1055ED00F80808E4F6A812F608F6E5122407F9A85B
:1055FD0012E6FE08E6FFC3099719E76480F8EE642A
:10560D0080985037E5122404F8CBE6CB08E6FA086B
:10561D00E6F98F828E83120721A812080866FFE52E
:10562D00122403F8EFF6E69048A393A8120808F6A3
:10563D00A8120806E61870B20680AFA8120808E690
:01564D00FF5D
:07564E00E5122409F5122208
:0B621600ED6F7817F6E69048A393FFA9
:01622100225A
:0300A300025C31CB
:105C3100C0E0C083C082C0D0E8C0E0EEC0E0EFC0E9
:105C4100E0E59830E1055398FDD230E59830E02445
:105C51007869E62401FFE433FEEF64404E70028070
:105C6100107869E60624D8F582E43402F583E599D3
:105C7100F05398FED0E0FFD0E0FED0E0F8D0D0D0D5
:065C810082D083D0E03266
:0A5419008B498A4A894B8C4C8D4D5B
:10542300E47869F6758401D284E54E24FF929BE407
:105433007818F67818E6C3954DE54C6480F87480C7
:05544300985060C2302A
:0D544800754F1475501300D550FCD54FF66C
:10545500E54D24FFFFE54C34FFFE7818E66F70013B
:10546500EE701EC2ACAB49054BE54BAA4A7002056E
:105475004A14F9120708F5993030FDC284D2AC8080
:1054850016AB49054BE54BAA4A7002054A14F912B9
:105495000708F5993030FD7F01125FF17818068015
:0554A50090C284AF4D30
:0154AA0022DF
:0A5164008B418A4289438C448D453B
:10516E001261A278191209B5E47818F61261A2EC50
:10517E00C0E0EDC0E0EEC0E0EFC0E0781912096CBF
:10518E00CBEFCBCAEECAC9EDC9C8ECC8D0E0FFD090
:10519E00E0FED0E0FDD0E0FCC3EF9BFFEE9AFEED0B
:1051AE0099FDEC98FCE47B01FAF9F8C31208DE5085
:1051BE00037F00227869E6FED3940040539002D814
:1051CE00E0FDB478037F0122ED54F8647860037F2C
:1051DE0000229002D8E0540724027818F66E703040
:1051EE007869E6D39545E5446480F8748098400666
:1051FE00AE44AF4580067869E6FF7E00A843AC4218
:10520E00AD417B017A0279D81206E27818E6FF22C8
:08521E007F01125FF102517AD9
:07000300E47869F6D2302217
:105D7E00EF7025F5847598D0F584759115F58475B9
:105D8E00C90875CBFFED9049A293F5CA75C804E416
:105D9E00F584D2ACC2BC80267584017598D0E4F52A
:105DAE0084E589540F4420F589758E02ED9049AC37
:105DBE0093F58DD28E43E74043F740120003D2AFE6
:015DCE0022B2
:105933009003181209E60000000090031C1209E608
:10594300000000009002CF7464F0E47818F6781831
:10595300E6FFC394025043EF25E025E024D0F5820F
:10596300E43402F583E4F0EF25E025E024D1F58269
:10597300E43402F583E4F0EF25E025E024D2F58258
:10598300E43402F583E4F0EF25E025E024D3F58247
:0A599300E43402F583E4F00680B46A
:01599D0022E7
:10610B00D2AFD2A9C2BBE4F584E589540F4401F5A3
:0F611B0089758E02758CAFE4F58AD28C025933E8
:024AB4001512D9
:104AB600A812E4F6A812E6FFC394024003024BA331
:104AC600EF25E025E024D3F582E43402F583E0FF08
:104AD600D394005003024B78E625E025E024D1F577
:104AE60082E43402F583E06003024B78EF30E0198C
:104AF600E6FF25E025E024D3F582E43402F583E0E1
:104B0600D3940140047D0080067D01A812E6FF12C1
:104B16005857A812E6FF25E025E024D3F582E434B1
:104B260002F583E0B401057D01125857A812E6FF8D
:104B360025E025E024D3F582E43402F583E014F081
:104B4600EF25E025E024D3F582E43402F583E06026
:104B560021E6FF25E025E024D2F582E43402F58340
:104B6600E0FEEF25E025E024D1F582E43402F5836A
:104B7600EEF0A812E6FF25E025E024D1F582E43424
:104B860002F583E06011EF25E025E024D1F582E40B
:0D4B96003402F583E014F0A81206024ABABA
:034BA300051222D6
:03000B0002537E1F
:10537E00C0E0C0F0C083C082C0D0E8C0E0E9C0E0A9
:10538E00EAC0E0EBC0E0ECC0E0EDC0E0EEC0E0EF64
:10539E00C0E0758CAF900318E0FCA3E0FDA3E0FE27
:1053AE00A3E02401FFE43EFEE43DFDE43CFC90035B
:1053BE00181209C19002CFE014F0E0702590031C82
:1053CE00E0FCA3E0FDA3E0FEA3E02401FFE43EFE2B
:1053DE00E43DFDE43CFC90031C1209C19002CF7425
:1053EE0064F0124AB41260E9D0E0FFD0E0FED0E0E3
:1053FE00FDD0E0FCD0E0FBD0E0FAD0E0F9D0E0F850
:0B540E00D0D0D082D083D0F0D0E032AC
:105FC4001512A812EDF61512A812EFF6A812E6FFA4
:105FD400C39402501308E6FEEF25E025E024D0F533
:0D5FE40082E43402F583EEF005120512226E
:1054AB0015121512A812EAF608EBF61512A812ED52
:1054BB00F61512A812EFF6A812E6FFC39402506A73
:1054CB00EF25E025E024D3F582E43402F583E07088
:1054DB0059E6FB25E025E024D1F582E43402F5837F
:1054EB00E0704708E625E004FFA812E6FA25E02560
:1054FB00E024D3F582E43402F583EFF00808E6FEEE
:10550B0008E6FF7C007D0A1207E9EA25E025E02486
:10551B00D2F582E43402F583EFF0EB25E025E024AD
:10552B00D1F582E43402F583E4F0E5122404F5129C
:01553B00224D
:0E5857001512A812EDF61512A812EFF6151292
:10586500A81208E6FFC394025024EF25E025E024A2
:10587500D0F582E43402F583E06013A8120808E647
:1058850070047F0180027F00A8120808EFF6A812B5
:10589500A68475840FA81208E6FF700BA8120808E5
:1058A500E624FF9286800DEFB40109A8120808E6E8
:0958B50024FF9287A812E6F58495
:0758BE00051205120512227C
:1061A200C2AF900318E0FCA3E0FDA3E0FEA3E0FF72
:0261B200D2AF6A
:0161B40022C8
:1061B500C2AF90031CE0FCA3E0FDA3E0FEA3E0FF5B
:0261C500D2AF57
:0161C70022B5
:105FF1001512A812EFF6A812E67005786BF608F6EE
:10600100302E16786AE675F064A4FFC3786CE69FBB
:0C60110018E695F0500375FFA50512225B
:10612A00D22EE4786BF608F6EF786A6003F68002FE
:0F613A00760A75FF0775FFA5E4F58475EF04225B
:1061C800C22EE4786BF608F6786A76FF75FFDE75FE
:0361D800FFAD22F6
:1060E900786C06E618700106302E16786AE675F0A7
:1060F90064A4FFC3786CE69F18E695F0500375FF1A
:02610900A522CD
:046048008E438F44B0
:10604C00E4F545F546C3E5469544E54595435016BC
:10605C007FE87E031259B17F01125FF10546E546D8
:06606C0070E3054580DF32
:01607200220B
:10599E0043A0F075840F43A60FC290C294D2957F98
:0359AE00017E0077
:0459B1008E658F660A
:1059B500D3E56694FAE5659400500EEFD394004064
:1059C500407E1600DEFD1F80F2856567856668D31B
:1059D500E56894FAE567940040157FFA7E00125950
:1059E500B174062568F56874FF3567F56780E0D3FF
:1059F500E5669400E56594004007AF68AE67125907
:015A0500B1EF
:015A0600227D
:105A0700754F007550007551497B007A0079477DC5
:015A1700028C
:085A18008B4B8A4C894D8D4E29
:105A20007F01125FF1AB4FAA50A95112081F240049
:105A3000FFE5F034E0FE854B52854C53854D54E430
:105A4000FDEDC3954E501BEF2DF582E43EF583E44A
:105A500093AB52AA53A9548D827583001207600D2F
:0F5A600080DFAB4FAA50A951E4854EF0020882B7
:10522600754112754234754900754A00754B437BCA
:07523600007A0079417D02BE
:08523D008B458A4689478D4824
:105245007880E664F160030252DA1261C8C2AFE405
:10525500F58443B701758F01AB49AA4AA94B1208DA
:105265001F2400FFE5F034E07818F608EFF6AA46AB
:10527500A947781CA64508C6EAC608C6E9C6E47863
:105285001AF6781AE6C395485032781CCBE6CB0857
:105295000806E618CAE6CA70010614F91207087866
:1052A5001BF6E6FF78180806E618CCE6CC70010672
:1052B50014F5828C83EFF0781A0680C6E4F58F53D7
:1052C500B7F0AB49AA4AA94B8548F0120882D2AF7C
:0552D500E4FF12612A54
:0152DA0022B1
:105DCF007880E664F17046C2AF1261C8E4F584438F
:105DDF00B701758F03781976E008F67818F67819F9
:105DEF00E6FE08E6F5828E83E4F07F01125FF1781C
:105DFF001AE426F618740236F61806E6C39408401D
:0D5E0F00DDE4F58F53B7F0D2AFFF12612A2A
:015E1C002263
:1052DB00125DCFE4F543F544F549754A00754B4330
:1052EB00FB7A00798D7D1612523D125226E4F54061
:1052FB00E540C3786F965073E4F53FAB0CAA0DA94C
:10530B000E75F020E53FA4F58285F083120721602E
:10531B0056E53F75F020A429F9EA35F0FA90000D17
:10532B00120A27788AE68540F0A429F9EA35F0FAC3
:10533B00EBC0E0EAC0E0E9C0E0AB0CAA0DA90E752A
:10534B00F020E53FA4F58285F083120721FD754916
:10535B0000754A00754B43D0E0F9D0E0FAD0E0FB82
:10536B0012523D053F809405408085125226E47809
:02537B0080F6BA
:01537D00220D
:024C97008F4349
:104C9900E4F549F54AF546F54F755000755149FB5C
:104CA9007A00798D7D16125A18125A07E54864342C
:104CB9007004E54764127003434601E4F545E54590
:104CC900C3786F964003024D6AE4F544AB0CAA0D14
:104CD900A90E75F020E544A4F58285F08312072119
:104CE900607AE5436054E54475F020A429F9EA3572
:104CF900F0FA90000D120A27788AE68545F0A42972
:104D0900F9EA35F0FAEBC0E0EAC0E0E9C0E0AB0C43
:104D1900AA0DA90E75F020E544A4F58285F0831249
:104D29000721FD754F00755000755149D0E0F9D044
:104D3900E0FAD0E0FB125A18801DAB0CAA0DA90E9F
:104D490075F020E544A4F58285F083120721254AF0
:104D5900F54AE43549F5490544024CD50545024C67
:104D6900C7125A07E54864347004E54764127003B2
:054D7900434602AF46B5
:014D7E002212
:0258C5008F63EF
:1058C700302F6812599ED296E4F5647F0A7E001243
:1058D70059B130A7090564E564C394C840EDC29681
:1058E7001259ADC295D29075840F75A6FF1259ADA6
:1058F700E56354F0FFE5A054014FF5A0A21D929473
:105907001259ADD2961259ADC2961259ADE563C47C
:1059170054F0FFE5A054014FF5A0A21D929412592F
:0B592700ADD2961259ADC2961259ADD8
:015932002252
:105F67008F4353A00FE54354F042A0D2961259AD88
:105F7700C2961259AD53A00FE543C454F042A0D2C4
:105F8700961259ADC2961259AD7F647E000259B17F
:1057E300E47818F608F6C296C295C29475840F75CC
:1057F300A6FF43A503D290D29153A00143A020D288
:10580300967F01FE1259B1C2967F017E0012604855
:105813007F20125F6712599ED2967F647E001259D1
:10582300B130A703C22F22D22FC21D7F241258C525
:10583300C21D7F0B1258C5C21D7F201258C5C21D41
:105843007F0C1258C5C21D7F011258C5C21D7F06A9
:035853001258C523
:01585600222F
:0D620900C21D7F011258C5E4FDFF02617B3C
:1061DB00EF6006C21D7F0F8004C21D7F0C1258C5D5
:0161EB002291
:10617B00ED5403C43354E0FEEF541F44804EFFC272
:04618B001D0258C5D4
:106165008F62E562640D600BE562640A6005D21D0D
:066175001258C5AF6222C2
:10609D008B0F8A108911AB0FAA10A9111207086076
:1060AD00150511E5117002051014F9120708FFD23C
:0760BD001D1258C580E0220E
:1037E700202020202020202020200025622A62641B
:1037F7000025622A62750025622A640025622A75FF
:103807000025622A2E622A660025622A6C6400253A
:10381700622A6C7500253262753A257300202020D4
:103827002020202020004E6F207661726961626C33
:10383700657320646566696E65640020202020201A
:10384700202020202020202020202020202000456C
:10385700534320454E5445522020202D2020202020
:103867002B20200045534320454E5445522020200D
:103877002D20202020202B200045534320454E5447
:10388700455220202000455343202020202020207F
:103897002020002020202020002000506172616D30
:1038A7006574657273207772697474656E00746FDE
:1038B70020666C617368206D656D6F72792E00F4F8
:1038C70070000000F76E000000FA8F000000FD6D29
:1038D7000000000000000000036B000000064D0020
:1038E700000009470000000C5400000063000000BE
:1038F70000016D0000000267000000037300000074
:10390700046D000000056800000006410000000784
:103917004B0000000880430000098046000014485F
:103927007A00001550610000166261000017570009
:103937000000185600000019B50000001A540000D6
:10394700001B6C2F73001C52504D001D46000000D9
:103957001E4A0000005A250000005B52504D005CD3
:10396700636E74005D7800000000000000000235FF
:103977000000004E6F64652041647200008D0100F5
:10398700000000000000003F80000000000002353A
:10399700000000477270204164720000008F010030
:1039A700000000000000003F8000000000000A380F
:1039B70000000054696D650000000001034A010022
:1039C700000000000000003F8000000000000A38EF
:1039D700000000446174650000000001033A010023
:1039E700000000000000003F8000000000000032DF
:1039F700000004466C6173680000000000000000CE
:103A0700000000000000000000000000000000327D
:103A17000000045265626F6F740000000000000030
:0E3A2700000000000000000000000000000091
:0A5B2100C19EC126C125C11FC1208D
:06326A008B408A418942FD
:103270009000011207216438706085434985444AF3
:1032800085454BF54C754D0A7B017A03792E125C0E
:10329000DB7B017A03792E12000EC3EF940AEE64F1
:1032A0008094805032E490035CF07B017A03792EA5
:1032B00012000EC3740A9FFFE49EFE90035CE0C3FD
:1032C0009FEE6480F8748098500D7F2012616590A5
:1032D000035CE004F080D3023531E490032EF0ABC0
:1032E00040AA41A9429000021207216068E49003BD
:1032F0005CF090035CE075F005A424C6F582E4342C
:1033000038F583E493FF64636019AB40AA41A94296
:10331000900002120721FEEF6E600890035CE0044B
:10332000F080CF90035CE0FF75F005A424C6F58221
:10333000E43438F583E493601CEF75F005A424C7EA
:10334000F9743835F07549FFF54A894B7B017A03EA
:10335000792E125B2CAB40AA41A9429000011207C2
:10336000216066E490035CF090035CE075F005A4D6
:1033700024F8F582E43438F583E493FF6019AB4018
:10338000AA41A942900001120721FEEF6E60089049
:10339000035CE004F080D190035CE0FF75F005A4CD
:1033A00024F8F582E43438F583E493601CEF75F07B
:1033B00005A424F9F9743835F07549FFF54A894BAD
:1033C0007B017A03792E125B2C7B017A03792E1212
:1033D000000E90035DEFF0AB40AA41A9421207082E
:1033E00014601D14606424FE700302349A24046087
:1033F000030235317BFF7A3779E71260730235318A
:10340000AB40AA41A94290000412072190035D300D
:10341000E11CE0FFC3740A9FF549AB43AA44A945E8
:10342000120708F54A7BFF7A3779F202352EE0FF62
:10343000C3740A9FF549AB43AA44A945120708F58E
:103440004A7BFF7A3779F802352EAB40AA41A94270
:1034500090000412072190035D30E11FE0FFC37468
:103460000A9FF549AB43AA44A94512081FF54B85AD
:10347000F04A7BFF7A3779FE02352EE0FFC3740AEB
:103480009FF549AB43AA44A94512081FF54B85F0A7
:103490004A7BFF7A38790302352EAB40AA41A94214
:1034A00090000412072130E03390035DE0FFC37405
:1034B0000A9FF549900010120721FF600280027FE9
:1034C000038F4AAB43AA44A9451209028F4E8E4D81
:1034D0008D4C8C4B7BFF7A3879088052AB40AA41E7
:1034E000A94290000412072190035D30E121E0FF22
:1034F000C3740A9FF549AB43AA44A9451209028F38
:103500004D8E4C8D4B8C4A7BFF7A387910801FE0B2
:10351000FFC3740A9FF549AB43AA44A945120902A7
:103520008F4D8E4C8D4B8C4A7BFF7A387916122B3F
:0A353000477B017A03792E126073C5
:01353A00226E
:0D142600900355E0FBA3E0FAA3E0F97DFF81
:101433008D438B408A418942900001120721643811
:101443007003021C37AB40AA41A94212070824FECD
:10145300700302169824FE70030218F1240360033C
:10146300021C3790000412072120E103021552AB3E
:1014730040AA41A942900019120985C000C001C0C9
:1014830002C003AC43EC1203BBD003D002D001D0A3
:101493000012019EC004C005C006C007900320E0EF
:1014A300FC1203BBD003D002D001D0001200AD1256
:1014B30003EF900320EFF0AB40AA41A9429000153F
:1014C3001209229000111209851203447003021CB1
:1014D30037AB40AA41A942900011120922C004C0AF
:1014E30005C006C007900320E0FC1203BBA804A9B3
:1014F30005AA06AB07D007D006D005D004120344D3
:101503005014AB40AA41A9429000111209221203C0
:10151300EF900320EFF0AB40AA41A94290001512CF
:101523000922C004C005C006C007900320E0FC12D6
:1015330003BBA804A905AA06AB07D007D006D005AC
:10154300D00412034460025003021C37021683E5E1
:1015530043F4704CAB40AA41A942900011120922F6
:10156300C004C005C006C007900320E0FCE41203DA
:10157300BBA804A905AA06AB07D007D006D005D09F
:1015830004120344701AAB40AA41A94290001512F9
:1015930009229000111209851203446003021C37CB
:1015A300AB40AA41A942900019120985C000C001AD
:1015B300C002C003AC43EC1203BBD003D002D00182
:1015C300D00012019EC004C005C006C007900320CE
:1015D300E0FCE41203BBD003D002D001D000120020
:1015E300AD1203EF900320EFF0AB40AA41A9429064
:1015F3000015120922900011120985120344700389
:10160300021C37AB40AA41A942900011120922C023
:1016130004C005C006C007900320E0FCE41203BB2E
:10162300A804A905AA06AB07D007D006D005D004A5
:101633001203445014AB40AA41A94290001112096D
:10164300221203EF900320EFF0AB40AA41A942908E
:101653000015120922C004C005C006C0079003206C
:10166300E0FCE41203BBA804A905AA06AB07D00754
:10167300D006D005D00412034460025003021C3785
:10168300AB40AA41A9429000151209221203EF9020
:101693000320EFF022AB40AA41A9429000041207B5
:1016A3002120E103021796900019120985C000C09A
:1016B30001C002C003AC43EC1203BBD003D002D081
:1016C30001D00012019EC004C005C006C0079003EC
:1016D30020E0FCA3E0FDEC1203B6D003D002D0015E
:1016E300D0001200AD1203EF900320EEF0A3EFF051
:1016F300AB40AA41A9429000151209229000111291
:1017030009851203447003021C37AB40AA41A94266
:10171300900011120922C004C005C006C00790033F
:1017230020E0FCA3E0FDEC1203B6A804A905AA0679
:10173300AB07D007D006D005D0041203445017AB33
:1017430040AA41A9429000111209221203EF90030B
:1017530020EEF0A3EFF0AB40AA41A942900015128E
:101763000922C004C005C006C007900320E0FCA303
:10177300E0FDEC1203B6A804A905AA06AB07D0073F
:10178300D006D005D00412034460025003021C3774
:101793000218D9E543F4704FAB40AA41A942900027
:1017A30011120922C004C005C006C007900320E03F
:1017B300FCA3E0FDE41203B6A804A905AA06AB073F
:1017C300D007D006D005D004120344701AAB40AA48
:1017D30041A94290001512092290001112098512A5
:1017E30003446003021C37AB40AA41A9429000198D
:1017F300120985C000C001C002C003AC43EC120350
:10180300BBD003D002D001D00012019EC004C0059A
:10181300C006C007900320E0FCA3E0FDE41203B67A
:10182300D003D002D001D0001200AD1203EF900319
:1018330020EEF0A3EFF0AB40AA41A94290001512AD
:1018430009229000111209851203447003021C3708
:10185300AB40AA41A942900011120922C004C0055D
:10186300C006C007900320E0FCA3E0FDE41203B62A
:10187300A804A905AA06AB07D007D006D005D00453
:101883001203445017AB40AA41A942900011120918
:10189300221203EF900320EEF0A3EFF0AB40AA4136
:1018A300A942900015120922C004C005C006C00752
:1018B300900320E0FCA3E0FDE41203B6A804A9050D
:1018C300AA06AB07D007D006D005D00412034460A4
:1018D300025003021C37AB40AA41A94290001512E3
:1018E30009221203EF900320EEF0A3EFF022AB40A6
:1018F300AA41A94290000412072120E0030219B370
:10190300900320E0F8A3E0F9A3E0FAA3E0FBC00012
:10191300C001C002C003AB40AA41A9429000191202
:101923000985C000C001C002C003AC43EC1203BB75
:10193300D003D002D001D00012019ED003D002D038
:1019430001D0001200AD9003201209C1AB40AA419F
:10195300A942900011120922900320E0F8A3E0F9B4
:10196300A3E0FAA3E0FB1203445012AB40AA41A93F
:10197300429000111209229003201209C1AB40AA20
:1019830041A942900015120922900320E0F8A3E038
:10199300F9A3E0FAA3E0FB12034460025003021C24
:1019A30037AB40AA41A942900015120922021C310B
:1019B300AB40AA41A94290000412072120E103028F
:1019C3001ACE900019120985C000C001C002C003DD
:1019D300AC43EC1203BBD003D002D001D000120100
:1019E3009EC004C005C006C007900320E0FCA3E02E
:1019F300FDA3E0FEA3E0FFEC1203B1D003D002D0BD
:101A030001D0001200AD1203EF9003201209C1AB05
:101A130040AA41A94290001512092290001112090F
:101A2300851203447003021C37AB40AA41A94290BC
:101A33000011120922C004C005C006C0079003208C
:101A4300E0FCA3E0FDA3E0FEA3E0FFEC1203B1A8DA
:101A530004A905AA06AB07D007D006D005D0041207
:101A630003445015AB40AA41A94290001112092228
:101A73001203EF9003201209C1AB40AA41A942907F
:101A83000015120922C004C005C006C00790032038
:101A9300E0FCA3E0FDA3E0FEA3E0FFEC1203B1A88A
:101AA30004A905AA06AB07D007D006D005D00412B7
:101AB300034460025003021C37AB40AA41A9429081
:101AC30000151209221203EF021C31E543F470558D
:101AD300AB40AA41A942900011120922C004C005DB
:101AE300C006C007900320E0FCA3E0FDA3E0FEA333
:101AF300E0FFE41203B1A804A905AA06AB07D007C7
:101B0300D006D005D004120344701AAB40AA41A9F1
:101B13004290001512092290001112098512034404
:101B23006003021C37AB40AA41A942900019120975
:101B330085C000C001C002C003AC43EC1203BBD09C
:101B430003D002D001D00012019EC004C005C0061C
:101B5300C007900320E0FCA3E0FDA3E0FEA3E0FFA9
:101B6300E41203B1D003D002D001D0001200AD12B1
:101B730003EF9003201209C1AB40AA41A942900090
:101B830015120922900011120985120344700302F1
:101B93001C37AB40AA41A942900011120922C0048C
:101BA300C005C006C007900320E0FCA3E0FDA3E04E
:101BB300FEA3E0FFE41203B1A804A905AA06AB073C
:101BC300D007D006D005D0041203445015AB40AA69
:101BD30041A9429000111209221203EF900320122F
:101BE30009C1AB40AA41A942900015120922C004C1
:101BF300C005C006C007900320E0FCA3E0FDA3E0FE
:101C0300FEA3E0FFE41203B1A804A905AA06AB07EB
:101C1300D007D006D005D00412034460174015AB9B
:101C230040AA41A9429000151209221203EF900322
:051C3300201209C1228E
:105EAE008F40E92405F9E43AFA782E7C037D017ED1
:105EBE00007F081206E2E4900336F0900334E0FF10
:105ECE006007900333F0E4A3F0854049754A0175ED
:105EDE004B03754C2E7BFF7A38791C122B477BFFB8
:075EEE007A38792402607389
:1023C000124BA6EF6003D21E22301E40E490032D74
:1023D000F09003251209E60000000090032912097D
:1023E000E600000000C221C222C223C224E49003FE
:1023F0005BF01261A2E47B2C7A01F9F8C31208DECB
:102400004003022AE4C21ED213123E7A20261EC2C4
:1024100013123E7A90035BEFF07003022AD4D226A7
:10242000E064026003022AD4D225022AD4302512A5
:1024300090033A742DF0E4A3F090034A742DF0E475
:10244000A3F090035530251374FFF0A37439F0A363
:102450007475F09003597405F08013E50CF0A3E552
:102460000DF0A3E50EF07882E614900359F0900386
:1024700059E0FFC394035005E4A3F0801B90032DA3
:10248000E0FE7002800EEE90032DB50705E024FEFD
:102490008002E01490035AF07882E670142025112F
:1024A000FDFF12617B7BFF7A38792D122B470225C5
:1024B000FAE4900358F0900358E0FDC394034003FE
:1024C0000225FAE4FF12617B900358E0FF90035A63
:1024D000E02FFFE433FE90032DE07C00B50708EC0D
:1024E000B506047F1580027F20126165900358E0D5
:1024F000FD7F0112617B900358E0FF90035AE02FAB
:10250000FFE433FE900359E0FDD3EF9D7480F86E35
:1025100098400C7BFF7A387942122B470225F190C4
:102520000358E0FE90035AE0FD2EFFC007EEFFEDDA
:102530002FFFE433FEEF7805C333CE33CED8F9FF57
:10254000900355E0FBA3E0FAA3E02FF9EA3EFAD0AE
:1025500007125EAE900358E0FD7F0A12617B301FC8
:1025600040900358E0FF90035AE02FFFE433FE90C1
:10257000032DE07C00B50729ECB50625EF7805C3EF
:1025800033CE33CED8F9FF900355E0FBA3E0FAA396
:10259000E02FF9EA3EFA7543017544037545208042
:1025A0004D900358E0FF90035AE02FFFE433FEEF15
:1025B0007805C333CE33CED8F9FF900355E0FBA3A3
:1025C000E0FAA3E02FF9EA3EFAC003C002C001908E
:1025D0000355A3E0FAA3E02FF9EA3EFA90000D12AA
:1025E0000A278B438A448945D001D002D003123296
:1025F0006A900358E004F00224B690032DE075F0D1
:1026000020A430250F2475F9743935F0FA9003555C
:1026100074FF800D250EF9E50D35F0FA900355E5B0
:102620000CF0A3EAF0A3E9F030205A7D03E4FF1296
:10263000617B7BFF7A387956126073900324E075D2
:10264000F003A4240DFF90035AE0FE90032DE0C395
:102650009EFD12617B20090A302107C220E4FF128F
:1026600061DB200A03022AD4302203022AD4900319
:1026700024E004F0E064036003022AD4C220FF12C5
:1026800061DB022AD4201F030228497D03E4FF12E4
:10269000617B7BFF7A38796B12607390035AE0FF9D
:1026A00090032DE0C39FFD7F1312617B20090A3048
:1026B0002107C21FE4FF1261DB300A53202250C2FF
:1026C0001FE4FF1261DB900355E0FBA3E0FAA3E0F7
:1026D000F9120708FF7E00900355A3A3E090000DB8
:1026E000120A27A801AC02AD037B017A03792012FC
:1026F00006E230251290032DE0FF6003B40110D2F2
:1027000027788076F1800890032DE0FF1260C430B6
:102710000B0F20230C1214261261A290032512091C
:10272000C1300B2D1261A2A804A905AA06AB07901F
:102730000325E0FCA3E0FDA3E0FEA3E02446FFE4C4
:102740003EFEE43DFDE43CFCD31208DE40031214DF
:1027500026300B3B1261A2A804A905AA06AB07907C
:102760000325E0FCA3E0FDA3E0FEA3E024F4FFEEDC
:102770003401FEE43DFDE43CFCD31208DE40109041
:102780000355E0FBA3E0FAA3E0F97DF71214332030
:102790000B0A9003251209E600000000300C1C20F3
:1027A0002419900355E0FBA3E0FAA3E0F97D0112A0
:1027B00014331261A29003291209C1300C3A12613C
:1027C000A2A804A905AA06AB07900329E0FCA3E090
:1027D000FDA3E0FEA3E02446FFE43EFEE43DFDE46D
:1027E0003CFCD31208DE4010900355E0FBA3E0FA56
:1027F000A3E0F97D01121433300C3B1261A2A8044E
:10280000A905AA06AB07900329E0FCA3E0FDA3E01D
:10281000FEA3E024F4FFEE3401FEE43DFDE43CFCC5
:10282000D31208DE4010900355E0FBA3E0FAA3E0CA
:10283000F97D09121433300C03022AD490032912B3
:1028400009E600000000022AD47D03E4FF12617B48
:102850007882E6D394005003302537900355E0FB8F
:10286000A3E0FAA3E0F9900019120922E4FBFAF9B7
:10287000F81203444014900355E0FBA3E0FAA3E0F0
:10288000F990000412072130E2087BFF7A38798042
:1028900080067BFF7A38798D1260737F1212616532
:1028A0007BFF7A38799A1260737F131261657BFF20
:1028B0007A3879A012607320090C302109C226C22F
:1028C00025D213123E7A200A030229B230220302D3
:1028D00029B27882E6D394004061900355E0FBA3CF
:1028E000E0FAA3E0F9120708FFD39404504DEF94E7
:1028F000004048900019120922E4FBFAF9F812038B
:10290000445038D21F900355E0FBA3E0FAA3E0F94E
:10291000120708FF7E0090000D120A2778207C0322
:102920007D011206E290035AE0FF90032DE0C39F61
:10293000FD7F1312617B7F011261DB30252A90033A
:102940002DE0FF64026004EFB4031DD220E4900385
:1029500024F090035AE0FF90032DE0C39FFD7F0D0C
:1029600012617B7F011261DB30253790032DE0641B
:1029700004702FD227788076F1126209E4FDFF12ED
:10298000617B7BFF7A3879A21260737D01E4FF12CC
:10299000617B7BFF7A3879B51260737FB87E0B124A
:1029A000604830250D90032DE0B40506E4F58475EC
:1029B000EF10300B2A20232790032DE070122025E2
:1029C000077882E614F0800E90032D7405F08006DF
:1029D00090032DE014F01261A29003251209C1307A
:1029E0000B481261A2A804A905AA06AB079003250B
:1029F000E0FCA3E0FDA3E0FEA3E02446FFE43EFEEE
:102A0000E43DFDE43CFCD31208DE401E90032DE0C3
:102A100070122025077882E614F0800E90032D7442
:102A200005F0800690032DE014F0200B0A9003259A
:102A30001209E6000000003025089003587406F0E3
:102A400080077882E6900358F0300C2520242290ED
:102A5000032DE02401FFE433FE900358E0FD7C00E9
:102A600012079490032DEDF01261A2900329120930
:102A7000C1300C431261A2A804A905AA06AB0790B5
:102A80000329E0FCA3E0FDA3E0FEA3E02446FFE46D
:102A90003EFEE43DFDE43CFCD31208DE4019900309
:102AA0002DE02401FFE433FE900358E0FD7C00128A
:102AB000079490032DEDF0200C0A9003291209E6EB
:102AC00000000000300B0D300C0A202507E49003B5
:102AD0002DF0D225A2099221A20A9222A20B9223C2
:042AE000A20C92248E
:012AE40022CF
:1000A60002045BE86480F8E933E83360110460F029
:1000B600ED33EC337009E8FCE9FDEAFEEBFF2204C0
:1000C60060DED3EB9FEA9EE99DE8C2E78CF0C2F7BB
:1000D60095F0400CE8CCF8E9CDF9EACEFAEBCFFB87
:1000E60012042685D0F05804700320D5B3E80470B6
:1000F600075002B2D502046592D5EC0460F7E4CC51
:10010600C0E0C398F8603B94186008400DD0E0FB4F
:1001160002043DE4FBFAC9FC8028E830E406E4C9A1
:10012600FBE4CAFCE830E305E4C9CACBFCE85407A3
:100136006010F8C3E913F9EA13FAEB13FBEC13FCAE
:10014600D8F130F52FC3E49CFCEF9BFFEE9AFEED51
:1001560099FDD0E0FBEF4E4D4C701222DB030204FA
:1001660062EC2CFCEF33FFEE33FEED33FDED30E7B2
:10017600EB02043DEF2BFFEE3AFEED39FDD0E0FB3E
:1001860050130BBB0003020465ED13FDEE13FEEFE7
:0801960013FFEC13FC02043D11
:10019E00EC4D6011E8497017ED33EC3304600DE45B
:1001AE00FCFFFEFD22E933E8330470F802045B1213
:1001BE00042658046009E4CC248150062850090214
:1001CE000465284003020462C0E0EB4A7044B98023
:1001DE0006D0E0FB020451EF4E701CBD8008EBFF11
:1001EE00EAFEE9FD80EBE98DF0A4FEE5F002028760
:1001FE00E9CDF9EAFEEBFFEF89F0A4FCE5F0CE893C
:10020E00F0A42EFFE435F0CD89F0A42DFEE435F0F8
:10021E008067EF4E7005BD80D780C3EF8BF0A4AC26
:10022E00F0EE8BF0A42CFCE435F0F8EF8AF0A42C61
:10023E00E5F038FCE433CB8DF0A42CFCE5F03BF874
:10024E00EE8AF0A42CFCE5F038F8E433CF89F0A464
:10025E002CFCE5F038CF3400CE89F0A42FFFE5F06A
:10026E003EFEE433C98DF0A42EFEE5F039CD8AF0C2
:10027E00A42FFFE5F03EFEE43DFD33D0E0FB50073A
:10028E000BBB000F020465EC2CFCEF33FFEE33FECC
:06029E00ED33FD02043DFA
:1002A400020465EC5D046005E85904700302045B14
:1002B400120426580460F6EC4860F2EC7004FDFE6B
:1002C400FF22C860DB2481C85009C398600250062D
:1002D4000204629850CAF582E9294B4A7005AB8240
:1002E40002045175F0007C1A7880C3EF9BEE9AEDFE
:1002F40099400DC3EF9BFFEE9AFEED99FDE842F0A5
:10030400DC23ACF0D0E0FFD0E0FED0E0FDAB8220F7
:10031400E7101BEB60BAEC2CFCEF33FFEE33FEED81
:1003240033FD02043DE803F830E705C0F075F00042
:10033400EF2FFFEE33FEED33FD40B830E7C280AA65
:1003440074F8CC6480CCC86480C8F582046043C36C
:10035400EB9FF5F0EA9E42F0E99D42F0E89C45F0FF
:1003640060305018E5825FFFE582F42B5582FB5024
:10037400210ABA001D09B90019088016E5825BFB41
:10038400E582F42F5582FF50090EBE00050DBD0015
:10039400010CC3EB9FF5F0EA9E42F0E99D42F0E8C0
:0D03A4009C45F06007CC4820E701B3EC2237
:1003B10075F020800E75F010800575F0087D007EC7
:1003C100007F003392D530D5031208BAEC334010C8
:1003D100EF33FFEE33FEED33FDEC33FCD5F0ED22D0
:0E03E100E5F0247EA2D513CC92E7CDCEFF220C
:1003EF00EDD2E7CD33EC3392D524814006E4FFFE06
:1003FF00FDFC22FCE4CFCECDCC24E0501174FF8065
:10040F00EDC3CC13CCCD13CDCE13CECF13CF047001
:07041F00F030D5DE0208BA3F
:102AE500E55D2449F8E6055D227846301B02784904
:102AF500E475F001120A170207082014EB7F2ED2A5
:102B0500148018EF540F2490D43440D4FF30180BA0
:102B1500EF24BFB41A0050032461FFE55E6002157F
:102B25005E0561E56170020560301B0D7846E47550
:102B3500F001120A17EF02074E0261657403D21BFA
:102B45008003E4C21BF55D8B468A478948E4F55E40
:102B5500F560F561E55E60077F20122B2080F57535
:102B65005FFFC215C214C216C217C219C21AC21C0F
:102B7500122AEEFF700D301B057F00122B31AF615D
:102B8500AE6022B4255FC2D5C218122AEEFF24D04A
:102B9500B40A00501A75F00A785E30D50508B6FFFC
:102BA5000106C6A426F620D5047002D21780D924C2
:102BB500CFB41A00EF5004C2E5D218022E1ED2156A
:102BC50080C6D21480C0D21680BCD2D580BAD219A4
:102BD50080B47F20122B202016077401B55E0040BB
:102BE500F1122AE5FF122B20022B59D21CD21A8092
:102BF50095122AE5FB122AE5FA122AE5F94A4B70E5
:102C05000679157A2F7BFF20162EE55E602A7E0059
:102C15008E8275830012072160060EEE655F70F0E7
:102C2500C2D5EBC0E0EAC0E0E9C0E0EE122E7ED0EE
:102C3500E0F9D0E0FAD0E0FB120708FF60AAEBC08C
:102C4500E0EAC0E0E9C0E0122B20D0E02401F9D091
:102C5500E03400FAD0E0FBE55F0460DCD55FD980A5
:102C650087D21680A2122E6160F7E55F700104120B
:102C75000470A95F600DE55F600914F55F122F0808
:102C8500EF60F3EA30E702F404C3995077EAF425DC
:102C95005F0430E701E404F55F800D122E6160C129
:102CA500EA055F255F120470EA785CF630E701E417
:102CB500255F04D55F0420190114122E7EE4C0E0BF
:102CC500122F08785CE6601320E70714F6122B082C
:102CD500802204F6D0E014C0E07F00122B08E55FE7
:102CE5006007122AFF155F800B301903122AFFD0E7
:102CF500E0022B59D0E00480C5122E6160A0E55F8B
:102D050004120470785CEAF6E55F2019026001049C
:052D15002404122E7ED3
:102D1A0074FF04C0E0122F08122B08E55F20190285
:102D2A006003122AFFD0E0B55FE87F45122B1278C4
:102D3A005CE67F2B30E7047F2DF404C0E0122B20E1
:102D4A00D0E075F00A84C0F0122B09D0E0122B09EA
:102D5A00022B59791080027908C21AC21C8008D243
:102D6A00D5790A8004790AC2D5E55F047002F55F55
:102D7A00E4FAFDFEFF122AE5FC7B08201513122A4D
:102D8A00E5FD7B1030140A122AE5FE122AE5FF7BC4
:102D9A0020EC3382D592D55013C3E43014069FFF3A
:102DAA00E49EFEE42015039DFDE49CFCE4CBF8C2FE
:102DBA0015EC700CCFCECDCCE824F8F870F3801760
:102DCA00C3EF33FFEE33FEED33FDEC33FCEB33FBA5
:102DDA00994002FB0FD8E9EB301505F8D0E0C4485A
:102DEA00B215C0E00AEC4D4E4F78207B0070C2EA63
:102DFA00B55F0040BCC0E0122E80D0F0D0E02015B4
:102E0A0004C4C0E0C4B215C0F0122B09D0F0D5F04A
:102E1A00EB022B59120A572BF6532D5D582BC74C30
:102E2A002BC3422D614F2D69442D69492BDC432D5B
:102E3A006F552CA0462CFE452C6A472F35502BCBBC
:102E4A002D2BCF2E2BF22B2BD3232BF0202F1E2A08
:102E5A002B8B4800002BEAE55FB4FF03755F06126F
:102E6A002AE5FC122AE5FD122AE5FE122AE5FF7878
:102E7A005502049F790AA2D5201714301909B910EE
:102E8A00020404B9080104A2D5201A025001042040
:102E9A0016689216B55E005034C0E07F20301719CC
:102EAA007F30A216721A7219500F122ED7C216C28A
:102EBA001AC219C21C7F30800F301903E9C0E01210
:102ECA002B20301903D0E0F9D0E0B55ECC301917C9
:102EDA007F30B9100C122B207F583018077F78806A
:102EEA0003B90803122B203016057F2D022B207FF1
:102EFA0020201CF87F2B201AF322921680CF7F0005
:102F0A00B4070050052455F8E6FF22286E756C6C4C
:102F1A002900D215122AE53015F8C215785E30D587
:102F2A000108F6022B8B2D50434958122AE5240337
:102F3A00B405004001E4902F3093122B11743A1219
:0A2F4A002B11D217755E04022D5DF5
:10042600E9D2E7C933E833F892D5EDD2E7CD33EC1C
:0704360033FC5002B2D52295
:10043D00EC30E7100FBF000C0EBE00080DBD000420
:10044D000BEB6014A2D5EB13FCED92E7FD2274FFCC
:10045D00FCFDFEFF22E480F8A2D574FF13FC7D8025
:03046D00E480EF39
:10047000F920E72824F950037907E4F42402FB1853
:10048000DBFDE624FB5014E9600DE4F618E604F603
:0F049000B40A08E4F6D9F57401F60A22C2D5229F
:10049F00ED33EC3392D5FA602AB4FF33EDC2E77B2C
:1004AF00FF60067A0479C4E4227A0479CD20D5045A
:1004BF007A0479C8224E614E002B494E46002D49D1
:1004CF004E4600E47A08F608DAFC7B00740722E84F
:1004DF00C0E0ECC0E0EDC0E0EEC0E0EFC0E0EA75D8
:1004EF00F010A4CAABF075F04DA42BFBE435F0FC73
:1004FF00EA2410FAEB34C5FBEC34D9FCEDC2E7FF6C
:10050F0075F056A4F42411C5F0F434C58FF0A42A65
:10051F00E5F03BE43CF620E7141205D2D0E0FFD023
:10052F00E0FED0E0FDD0E0FC1202A78014F404122C
:10053F0005D2D0E0FFD0E0FED0E0FDD0E0FC12010C
:10054F009ED0E0F8E6FAEDD2E7CD33EC332482FB10
:10055F00E4C3CF33CFCE33CECD33CD33DBF37B07F5
:10056F0075F00A846004F6081B0AE5F0F6088FF0B0
:10057F00740AA4FFACF08EF0740AA42CFEACF050F9
:10058F00010C8DF0740AA42CFDE435F0F608DBDEC7
:03059F00740722BC
:1005A2003F8000004120000042C80000447A000061
:1005B200461C400047C35000497424004B189680E3
:1005C2004CBEBC205A0E1BCA6753C21C749DC5AEDA
:1005D200FB60065407601C2323120600EB543860AC
:1005E200091205EC1205FB12019EECF8EDF9EEFA88
:1005F200EFCB22EB1205FB80F1543803241C90054B
:10060200A2FE93FC0EEE93FD0EEE930ECE93FF220E
:0300000002565550
:0C565500787FE4F6D8FD7581A202569C17
:10061200E709F608DFFA8046E709F208DFFA803ECA
:1006220088828C83E709F0A3DFFA8032E309F608B7
:10063200DFFA8078E309F208DFFA807088828C831F
:10064200E309F0A3DFFA806489828A83E0A3F608D3
:10065200DFFA805889828A83E0A3F208DFFA804CAD
:1006620080D280FA80C680D4806980F28033801084
:1006720080A680EA809A80A880DA80E280CA8033ED
:1006820089828A83ECFAE493A3C8C582C8CCC58365
:10069200CCF0A3C8C582C8CCC583CCDFE9DEE78035
:1006A2000D89828A83E493A3F608DFF9ECFAA9F0B4
:1006B200EDFB2289828A83ECFAE0A3C8C582C8CC0A
:1006C200C583CCF0A3C8C582C8CCC583CCDFEADE23
:1006D200E880DB89828A83E493A3F208DFF980CC85
:1006E20088F0EF60010E4E60C388F0ED2402B4047E
:1006F2000050B9F582EB2402B4040050AF23234525
:06070200822390066273E1
:10070800BB010689828A83E0225002E722BBFE02EF
:09071800E32289828A83E4932222
:10072100BB010CE58229F582E5833AF583E022508D
:1007310006E92582F8E622BBFE06E92582F8E222D7
:0D074100E58229F582E5833AF583E49322F1
:10074E00BB010689828A83F0225002F722BBFE018A
:02075E00F32284
:10076000F8BB010DE58229F582E5833AF583E8F0CF
:10077000225006E92582C8F622BBFE05E92582C87B
:02078000F22263
:10078200EF8DF0A4A8F0CF8CF0A428CE8DF0A42E8B
:02079200FE2245
:10079400BC000BBE0029EF8DF084FFADF022E4CC49
:1007A400F875F008EF2FFFEE33FEEC33FCEE9DEC12
:1007B400984005FCEE9DFE0FD5F0E9E4CEFD22ED58
:1007C400F8F5F0EE8420D21CFEADF075F008EF2FA2
:1007D400FFED33FD4007985006D5F0F222C398FD93
:0507E4000FD5F0EA2230
:1007E900C2D5EC30E709B2D5E4C39DFDE49CFCEE2B
:1007F90030E715B2D5E4C39FFFE49EFE120794C308
:10080900E49DFDE49CFC800312079430D507C3E402
:060819009FFFE49EFE2299
:10081F00BB010A89828A83E0F5F0A3E022500687A4
:10082F00F009E71922BBFE07E3F5F009E319228966
:0B083F00828A83E493F5F07401932299
:10084A00BB0110E58229F582E5833AF583E0F5F0EC
:10085A00A3E0225009E92582F886F008E622BBFEC9
:10086A000AE92582F8E2F5F008E222E5832AF5830F
:08087A00E993F5F0A3E99322D4
:10088200BB010789828A83020AA9500B09C5F02796
:10089200F7C5F01937F722BBFE0D09F8E325F0F38F
:1008A200C5F019E338F322F889828A83740193250B
:0808B200F0C5F0F8E4933822D0
:0E08BA00C3E49FFFE49EFEE49DFDE49CFC224F
:1008C800EB9FF5F0EA9E42F0E99D42F0EC6480C8A7
:0608D80064809845F02247
:1008DE00EB9FF5F0EA9E42F0E99D42F0E89C45F070
:0108EE0022E7
:1008EF00E8600FECC313FCED13FDEE13FEEF13FFE7
:0308FF00D8F1220B
:10090200BB010789828A83020ABF5005E9F80209FE
:100912006CBBFE05E9F8020ACB89828A83020AD7F8
:10092200BB010DE58229F582E5833AF583020ABF10
:100932005007E92582F802096CBBFE07E92582F817
:10094200020ACBE58229F582E5833AF583020AD7CA
:10095200BB010789828A830209C15005E9F80209AD
:0A096200B5BBFE05E9F8020B1022F8
:0C096C00E6FC08E6FD08E6FE08E6FF22B7
:0D097800E6FB08E6F908E6FA08E6CBF822EF
:10098500BB010DE58229F582E5833AF583020AE785
:100995005007E92582F8020978BBFE07E92582F8A8
:1009A500020AF3E58229F582E5833AF583020B0015
:0C09B500ECF608EDF608EEF608EFF6226E
:0C09C100ECF0A3EDF0A3EEF0A3EFF022A9
:1009CD00D083D082E493F608740193F608740293F1
:0909DD00F608740393F674047328
:1009E600A8828583F0D083D0821209FD1209FD12F8
:1009F60009FD1209FDE473E493A3C583C5F0C5831D
:100A0600C8C582C8F0A3C583C5F0C583C8C582C85A
:010A160022BD
:100A1700FAE6FB0808E6F925F0F618E6CA3AF622E0
:100A2700BB010DE58229F582E5833AF583020B25A3
:100A37005007E92582F8020B1CBBFE07E92582F85F
:100A4700020B2EE58229F582E5833AF583020B37FF
:100A5700D083D082F8E4937012740193700DA3A32E
:100A670093F8740193F5828883E473740293686042
:060A7700EFA3A3A380DF42
:10607300120708601CFF09E970010AC0E0EAC0E0EA
:10608300EBC0E0126165D0E0FBD0E0FAD0E0F9802C
:0A609300DF7F0A126165E4FEFF22C0
:105B2C008B468A4789488B4C8A4D894EAB46054833
:105B3C00E548AA477002054714F912070870ED747E
:105B4C00FF2548F54874FF3547F547AB49054BE54C
:105B5C004BAA4A7002054A14F9120708FFAB460516
:105B6C0048E548AA477002054714F9EF12074E7032
:085B7C00DAAB4CAA4DA94E2240
:105CDB008B468A478948E4F54EF54FE54D154DAE99
:105CEB004C7002154C4E6033AB49AA4AA94B1207B4
:105CFB0008FFAB46AA47A948054FE54FAC4E7002CB
:105D0B00054E14F5828C83EF120760EF60CD7401A2
:105D1B00254BF54BE4354AF54A80C0AB46AA47A95B
:025D2B0048220C
:10000E00E4FFFE120708600C0FEF70010E09E97095
:05001E00F20A80EF2250
:10614900E94A4B700122120708FF6D700122EF70B6
:0C61590004FBFAF92209E970ED0A80EA63
:100A7D00EF4E6012EF60010EEDBB010B89828A8390
:100A8D00F0A3DFFCDEFA2289F05007F709DFFCA99D
:0C0A9D00F022BBFEFCF309DFFCA9F022F4
:105661000261FBE493A3F8E493A34003F68001F203
:1056710008DFF48029E493A3F85407240CC8C3334A
:10568100C4540F4420C8834004F456800146F6DF19
:10569100E4800B0102040810204080905AD0E47E7F
:1056A100019360BCA3FF543F30E509541FFEE4930E
:1056B100A360010ECF54C025E060A840B8E493A3D5
:1056C100FAE493A3F8E493A3C8C582C8CAC583CA00
:1056D100F0A3C8C582C8CAC583CADFE9DEE780BEB8
:015B2B000079
:100AA900C5F0F8A3E028F0C5F0F8E58215827002D8
:060AB9001583E038F02275
:0C0ABF00E0FCA3E0FDA3E0FEA3E0FF22AA
:0C0ACB00E2FC08E2FD08E2FE08E2FF2267
:100AD700E493FC740193FD740293FE740393FF2265
:0C0AE700E0F8A3E0F9A3E0FAA3E0FB2292
:0D0AF300E2FB08E2F908E2FA08E2CBF82283
:100B0000E493F8740193F9740293FA740393FB224B
:0C0B1000ECF208EDF208EEF208EFF22221
:090B1C00E6FB08E6FA08E6F922FE
:090B2500E0FBA3E0FAA3E0F922D1
:090B2E00E2FB08E2FA08E2F922F8
:0C0B3700E493FB740193FA740293F9221A
:00000001FF
